:1000000000800020BD010000F1520000BD52000040
:10001000BD520000BD520000BD520000BD520000A4
:10002000BD520000BD520000BD520000F152000060
:10003000F1520000BD520000F1520000AD5200002C
:10004000F1520000F1520000F1520000F1520000A4
:10005000F1520000F1520000F1520000F152000094
:10006000F1520000F1520000F1520000F152000084
:10007000F1520000F1520000F1520000F152000074
:10008000F1520000F1520000F1520000F152000064
:10009000F1520000F1520000F1520000F152000054
:1000A000F1520000F1520000F1520000F152000044
:1000B000F1520000F1520000F1520000F152000034
:1000C000F1520000F1520000F1520000F152000024
:1000D000F1520000F1520000F1520000F152000014
:1000E000F1520000F1520000F1520000F152000004
:1000F000F1520000695C0000F15200002D62000026
:10010000F152000009670000F1520000F1520000B6
:10011000F1520000F1520000F1520000F1520000D3
:10012000F1520000110A0000410D0000F1520000E0
:10013000F1520000F1520000F1520000F1520000B3
:10014000F1520000F1520000F1520000F1520000A3
:10015000F1520000F1520000F1520000F152000093
:10016000F1520000116A0000F1520000F15200004B
:10017000F1520000F1520000F1520000F152000073
:10018000F1520000F1520000F1520000A94A0000B3
:10019000F1520000F1520000F1520000F152000053
:1001A000F1520000F1520000F1520000F152000043
:1001B000F1520000F1520000F1520000564B4CF297
:1001C000205210B51A804DF628121A8000BF00BFC9
:1001D00005F092F8514B4FF010621A60504A9A6045
:1001E000504ADA60A3F53043203B1A6812F480725B
:1001F00004D14D490A604FF4A8521A604B4B1A784B
:10020000110703D51A7842F008021A70484B2A22C7
:100210001A700023474A48499818884204D247492F
:10022000595899500433F5E7454A464B9A424FF0E6
:10023000000302D242F8043BF7E74349434A5958C6
:1002400099500433B3F5DE7FF7D1414B802103F899
:10025000011B40498B42F9D13F4B1A603F4B0A22A8
:100260001A70A3F5805324225A70A0221A709A792A
:100270009207FCD59A79D406FCD4394B9A7902F0CE
:100280000C02082AF9D103221A7140225A719A7974
:100290009006FCD5324B9A795106FBD5314A32494A
:1002A00011600221516020221A702D4B9B7903F0BE
:1002B0000C030C2BF9D12D4B2D4A1A602D4B2E4AD5
:1002C0001A6000225A60072243F8042C2B4AC3F814
:1002D0000C2D62B605F024FA134B1B68DA0705D51E
:1002E000274805F041F8274B274A1A60274B1B780F
:1002F0005B0609D5234C244A2368934204D1204845
:1003000005F032F80023236007F058FE04F0FAFFEE
:1003100007F098F9FEE700BF0E200540308004404A
:10032000823F04000100002B14D0034002D007409C
:1003300000E007406087FF1F7C88FF1F40B200007D
:100340007C88FF1F1C91FF1F000000000082FF1F20
:1003500000E400E05FE400E008ED00E0005006404B
:100360000040064044800440000003010480044033
:10037000C010050014E000E0FF760100000020201E
:1003800000DD68501CE00340A5C3945A00F007400C
:10039000FFFFFFFFFFFFFFFFFFFFFFFFFFFFFFFF6D
:1003A000FFFFFFFFFFFFFFFFFFFFFFFFFFFFFFFF5D
:1003B000FFFFFFFFFFFFFFFFFFFFFFFFFFFFFFFF4D
:1003C000FFFFFFFFFFFFFFFFFFFFFFFFFFFFFFFF3D
:1003D000FFFFFFFFFFFFFFFFFFFFFFFFFFFFFFFF2D
:1003E000FFFFFFFFFFFFFFFFFFFFFFFFFFFFFFFF1D
:1003F000FFFFFFFFFFFFFFFFFFFFFFFFFFFFFFFF0D
:10040000FFFFFFFFFFFFFFFFFFFFFFFFFEFFFFFFFD
:1004100010B5054C237833B9044B13B10448AFF33E
:1004200000800123237010BD7C88FF1F00000000A6
:1004300040B2000008B5064B1BB106480649AFF3B1
:1004400000800648036813B1054B03B1984708BD07
:100450000000000040B200008088FF1F7C88FF1F62
:10046000000000002DE9F04101210D2005F024F8E5
:100470006D4B6E4C6E4E20221A604FF4847007F064
:10048000E9F8054602F046FB2846256002F0D5FA59
:10049000FE2811D140F2DC5005F02CF9902007F035
:1004A000D9F8644904464FF4E13200F0FBFF3460B0
:1004B000306802F08BF8FBE723685F4993F8A200ED
:1004C00004F062FF5D4B4FF496721A605C4BC022E1
:1004D0001A602368012193F8A20004F0EDFF23685D
:1004E000402193F8A20005F003F80C2004F0BCFCB6
:1004F000082004F0E3FC40F2DC5005F0FBF8206833
:1005000002F05DFA430803F1376303F5D833B3FB18
:10051000F0F005F053F9206802F073FA20B1236877
:1005200093F8A00005F0F6F9206802F074FA430889
:1005300003F1376303F5D833B3FBF0F005F028FC83
:10054000206802F071FA430803F1B76303F55843DA
:10055000B3FBF0F005F0FEFE206802F05CFA054601
:10056000582007F077F82A463649374D074603F0FA
:10057000A7FD20682F6002F022FA8046582007F07D
:1005800069F842463149074603F0EAF8304B5820F3
:100590001F6007F05FF8074600F0ECFB2D4B2E497B
:1005A0001F60384600F052FD902007F053F82149B3
:1005B0004FF4E132074600F075FF2068376002F023
:1005C00033FA0746902007F045F83A462249064696
:1005D00000F068FF214B28681E6003F0D5FD2868F5
:1005E0001F4E03681B6A98473768286807F2FA5756
:1005F00003F096FD3368BB4204D2286803681B6A87
:100600009847F7E760210B4620680A4602F09BF9FD
:1006100000F0D8F923681B7E23B10120BDE8F0412A
:1006200004F044B9BDE8F08184F00F40B488FF1FA6
:100630009888FF1FE490FF1F0000A041A488FF1FBF
:100640009C88FF1FC490FF1FBC88FF1FB490FF1F32
:10065000B088FF1FAC88FF1FD490FF1FB888FF1F12
:100660000089FF1F2D4B834208BF08462C4B984240
:1006700010B51FD12B4C05F019F9206802F0DCFCF5
:10068000962005F037F8284B1868430803F13763C4
:1006900003F5D833B3FBF0F005F090F8206802F0D2
:1006A000B0F9002838D02368BDE8104093F8A000C6
:1006B00005F030B91D4B984215D105F0E1FB194BFF
:1006C000186802F0B9FC962005F014F8164B18686B
:1006D000430803F1376303F5D833B3FBF0F0BDE80B
:1006E000104005F055BB124B984215D105F09EFE07
:1006F0000C4B186802F0A0FC962004F0FBFF0A4B9C
:100700001868430803F1B76303F55843B3FBF0F0EF
:10071000BDE8104005F01EBE10BD00BFE490FF1FF5
:10072000B490FF1FB488FF1F0C91FF1FC490FF1FE0
:10073000D490FF1F1C4B1A684FF6E85101328A42D1
:1007400070B51A601D462EDD184C2368D3F8AC0036
:1007500003F0FCFE23680C2690FBF6F6986803F085
:10076000EBFEB0F5967F05DDB0F5167FA8BF4FF420
:10077000167001E04FF496700D4A23681268A0F5D8
:1007800096700A21414391FBF2F10A4A93F8A200C4
:100790001268514301F52071F6B291FBF6F104F0B5
:1007A000A7FE00232B6070BDA888FF1FB488FF1F21
:1007B000A488FF1F9C88FF1F0F4B1A68002A08DAC5
:1007C0000E49086801280DD00120086020200C493E
:1007D00007E007D00949086820B1002008600949EE
:1007E0002020086001324FF6E8518A42C8BF6FF0FE
:1007F00031021A60704700BFA088FF1F6087FF1F8B
:1008000084F00F4088F00F402DE9F74F634B644DA3
:100810001A68644C92F8BC20634F644E98468AB9BB
:10082000286801F0D3FE206801F0D0FE386803F09C
:1008300005FA306803681B6A9847FFF77BFFFFF7EC
:10084000BBFFE3E7386810B103689B6898473068DE
:1008500010B103689B689847286810B103689B68CB
:100860009847206810B103689B68984700F0C6F865
:10087000D8F800301B7E0BB104F086F9D8F80030B0
:10088000DFF8389193F8BC3003F0040203F002055E
:1008900002F0FF061AB125B92E46042502E04C46A7
:1008A00001E00426424CD90704D50DB9012500E02A
:1008B0000126404C1A0704D50DB9082500E008268A
:1008C0003D4C13F0160F04D00DB9162500E0162686
:1008D0003A4C3B4B93F800A000270AF0010A9B46D4
:1008E0000021D8F800000A46802302F02CF8022DDF
:1008F00001D0022E08D1BAF1000F05D19BF80030CB
:1009000013F0010F18BF01279BF800A00AF0010A9D
:10091000D9F8003029489B68984758B31FB1274839
:100920002146FFF79FFEFF210022D8F80000802318
:1009300002F009F8236821481F68D9F80030DB6805
:100940009847C1B22046B8470027E1E7CFB9002158
:10095000D8F80000FF22802301F0F5FFD9F800301D
:100960001A6823682046DB6801929847019AC1B251
:1009700012489047236820469B6898470028E5D195
:1009800007E04C45E3D120462146FFF76BFE0027E8
:10099000DDE7FFF7CFFEFFF70FFFA1E7B488FF1FEA
:1009A0009888FF1FB888FF1FB088FF1FBC88FF1FF3
:1009B000B490FF1FC490FF1FD490FF1FE490FF1F4F
:1009C000B090FF1F08B5094B4FF000721A604FF04E
:1009D00080621A60064B1B6893F82500054B18705F
:1009E00004F006FB044B01221A7008BD04E100E08C
:1009F000B488FF1FC088FF1FC288FF1F034B4FF042
:100A000000721A604FF080621A60704784E100E063
:100A100070B5B24C23780F2B00F28781DFE813F01A
:100A2000210036004B00600075008A009F00B40072
:100A3000C900DE001D013401010168014A011000F6
:100A4000A74D287804F01CFBA64B1B68D3F8AC20FC
:100A5000132101FB0200142690FBF6F2C3F8AC2030
:100A6000D8E09F4D287804F00BFB9E4B1B681A6B57
:100A7000452101FB0200462690FBF6F21A6393F82B
:100A80002500287004F0B4FA01234CE1944D287835
:100A900004F0F6FA934B1B685A6B452101FB0200E8
:100AA000462690FBF6F25A6393F82600287004F06D
:100AB0009FFA022337E18A4D287804F0E1FA894B46
:100AC0001B689A6B452101FB0200462690FBF6F25B
:100AD0009A6393F82700287004F08AFA032322E12E
:100AE0007F4D287804F0CCFA7E4B1B68DA6B4521E9
:100AF00001FB0200462690FBF6F2DA6393F8280029
:100B0000287004F075FA04230DE1754D287804F07F
:100B1000B7FA744B1B681A6C452101FB020046268C
:100B200090FBF6F21A6493F82900287004F060FA3A
:100B30000523F8E06A4D287804F0A2FA694B1B6897
:100B40005A6C452101FB0200462690FBF6F25A64DE
:100B500093F82A00287004F04BFA0623E3E0604D76
:100B6000287804F08DFA5F4B1B689A6C452101FBD5
:100B70000200462690FBF6F29A6493F82B00287048
:100B800004F036FA0723CEE0554D287804F078FAC1
:100B9000544B1B68DA6C452101FB0200462690FB92
:100BA000F6F2DA6493F82C00287004F021FA082396
:100BB000B9E04B4D287804F063FA4A4B1B681A6D74
:100BC000452101FB0200462690FBF6F21A6593F8D8
:100BD0002D00287004F00CFA0923A4E0404D287879
:100BE00004F04EFA3F4B1B685A6D452101FB020091
:100BF000462690FBF6F25A653B4A1178092907D937
:100C0000987B28700021117004F0F2F90C238AE01F
:100C10000131117093F82400287004F0E9F90023E1
:100C200081E02F4D287804F02BFA2E4B1B681A69AF
:100C3000632101FB0200642690FBF6F2597B1A61E6
:100C40002A4A52F83120012182F8801093F8950049
:100C5000287004F0CDF90A2365E0214D287804F0CE
:100C60000FFA204B1B68D3F89C2002EBC202104401
:100C70000A2190FBF1F2C3F89C2093F894002870AD
:100C800004F0B6F90B234EE0154D287804F0F8F97E
:100C9000144B1B68D3F8982002EBC20210440A21BF
:100CA00090FBF1F2C3F898201879287004F0A0F9AD
:100CB0000E2338E00A4D287804F0E2F9094B1B684E
:100CC0009A68312101FB0200322690FBF6F29A600D
:100CD000987B287004F08CF90D2324E0C288FF1F54
:100CE000C088FF1FB488FF1FC188FF1FC4AD00006C
:100CF000104D287804F0C4F90F4B1B685A69632122
:100D000001FB0200642690FBF6F2597B5A610B4A04
:100D100052F83120012182F8001193F8A8002870C0
:100D200004F066F90F23237070BD0220BDE8704007
:100D300003F018BCC088FF1FB488FF1FC4AD0000BB
:100D4000FFF766BE38B5044608460D4607F07DFA43
:100D5000236802465B6820462946984738BD38B567
:100D60000446FFF7EFFF0546204606F097FC2844AF
:100D700038BDFFFF38B5002504460571457180F880
:100D8000545004491422063007F07EFA25652046A7
:100D900038BD00BF908E00000079704790F8552054
:100DA000044B53F83220012382F880300371184637
:100DB000704700BFC4AD000038B5084B90F855200F
:100DC00053F832300124054683F800410A2004F02C
:100DD00091FC00232B71204638BD00BFC4AD00003C
:100DE0004079704706307047006D704738B504464B
:100DF000006803681B6A98472046FFF7DDFF94F8F8
:100E000056200E4B53F83230012583F880500A20CB
:100E100004F070FC2046FFF7C1FF2068084B202239
:100E20001A6003684FF416419B69984740F2EE2020
:100E300004F060FC84F8545038BD00BFC4AD00001D
:100E400084F00F4070B50446006803681B6A984739
:100E50002046FFF7B1FF94F856200E4B53F832307E
:100E6000012283F800210A2004F044FC2046FFF709
:100E700095FF2568084B20221A602B689E69074B56
:100E8000186801F0D1FD01462846B047002384F8D8
:100E9000543070BDC4AD000088F00F40B488FF1F0F
:100EA00010B58EB0322201A80C4607F0EDF90023F0
:100EB0003A2101A88DF8353007F0A8F9014608B9A4
:100EC000207003E02046013107F0B7F90EB010BDE5
:100ED0002DE9F84300250746884691460D702C46BB
:100EE0002E46386803689B68984748B3386803689B
:100EF000DB689847C0B20EB945282DD001360D28C1
:100F0000F6B203D1002308F8043009E009F1FF33F9
:100F10009C42F7D008F804000134E4B20025E0E771
:100F2000386803689B68984738B138680368DB689D
:100F300098470A2004F0DEFBF2E70120BDE8F883C1
:100F400001350A20EDB204F0D5FB312DC9D9201CA2
:100F500018BF0120BDE8F8833046BDE8F883FFFFE5
:100F600070B5044625460679FFF740FF002355F883
:100F70001A0B0E496371FFF7F2FE20462946322212
:100F8000FFF7A6FF38B128460949022207F065F9A4
:100F900008B9012300E0002363712046FFF752FFE8
:100FA00016B92046FFF708FF607970BDB68E0000C5
:100FB000B38E0000437970B50446F3B190F85460E5
:100FC0000EB9FFF713FF25460C4955F81A0BFFF72A
:100FD000C6FE322229462046FFF77AFF20462946E0
:100FE000FFF75EFFA01D2946142207F04DF926B930
:100FF0002046BDE87040FFF725BF70BDB98E0000E8
:10100000437970B50446EBB190F854600EB9FFF720
:10101000EDFE25460C4955F81A0BFFF7A0FE3222CB
:1010200029462046FFF754FF20462946FFF738FFA0
:10103000284606F0B1FF206526B92046BDE870407D
:10104000FFF700BF70BD00BFC28E000070B52B4D12
:1010500001600446286801F0F0FC032804D1212334
:1010600084F85530172306E00438012837D80323C5
:1010700084F85530182384F8563094F8560001212E
:1010800004F01AFA94F856201D4B53F8323001211F
:1010900083F8001194F8550004F00EFA2046FFF78B
:1010A0007DFE2046FFF75CFF637933B32046FFF7F0
:1010B0009DFE2046FFF7A4FF2046FFF77BFF20465A
:1010C000FFF7C0FE2046FFF769FE24682868236802
:1010D0009E6901F0A9FC01462046B0470DE00A20B8
:1010E00003F040FA074B063403F1140253F8041BD3
:1010F00044F8041B9342F9D170BD70BDB488FF1F42
:10110000C4AD0000CB8E0000F8B5437904460F460D
:1011100043B390F854600EB9FFF768FE25463A468F
:101120001149206806F0D0FA55F81A0B0F49FFF75D
:1011300009FE204629463222FFF7CAFE60B1284642
:101140000B49022207F089F830B9A01D3946142254
:1011500007F09AF8012500E0002516B92046FFF7B0
:1011600071FE2B461846F8BDDF8E0000B08E0000E1
:10117000B38E0000437970B504460D462BB390F84A
:1011800054600EB9FFF732FE2A4625461049206802
:1011900006F09AFA55F81A0B0E49FFF7D3FD2046D0
:1011A00029463222FFF794FE48B128460A49022216
:1011B00007F053F8D0F1010538BF002500E00546DF
:1011C00016B92046FFF73EFE2B46184670BD00BFFD
:1011D000A18E0000B08E0000B38E0000F8B54379F8
:1011E00004460F4623B390F854600EB9FFF7FEFD96
:1011F00025463A460F49206806F066FA55F81A0B5C
:101200000D49FFF79FFD204629463222FFF760FE79
:1012100040B128460949022207F01FF810B9276596
:10122000012500E0002516B92046FFF70BFE2B46EE
:101230001846F8BDEA8E0000B08E0000B38E0000A4
:10124000F8B5437904460F4600F11A050BB98376C9
:1012500015E090F854600EB9FFF7C8FD39462068D4
:10126000FFF770FD07492068FFF76CFD204629460F
:101270003222FFF72DFE16B92046FFF7E3FD284680
:10128000F8BD00BFB08E00000023012110B50A4652
:101290000446C3600361094B4FF4BF7003F096F935
:1012A000042120600122064B4FF4BF7003F08EF939
:1012B00042236060A360204610BD00BFF78E00008F
:1012C000088F00000A23034AB1FBF3F1B2FBF1F3EC
:1012D0008360704730D4050010B50446006806F0FE
:1012E0009BFE606806F098FE204610BD0369026808
:1012F000D154084A03691168426842F823105A1C05
:10130000B2F5BF7FA5BF6FF4BE729B180261036187
:10131000704700BF0089FF1FC26803699A42CABFB5
:10132000C2F5BF72C2EB0300D018704738B50D4646
:101330000446FFF7F1FF854204DB062003F012F9B3
:10134000002038BDE16823682944B1F5BF7FA8BFFC
:10135000A1F5BF71585C38BDC36800695A1E48BF0B
:1013600003F27D12131A5842584170470023C3609C
:101370000361704738B50D460446FFF7CDFF85423F
:1013800004DD0820BDE8384003F0ECB8E1682944EA
:10139000B1F5BF7FA8BFA1F5BF71E16038BDFFFF08
:1013A00038B50B4B1D6883680446ED1A2046FFF7DD
:1013B000B3FF00280ADDE268636853F82230AB42CD
:1013C00004D820460121FFF7D5FFEFE738BD00BF65
:1013D0000089FF1F014B0360704700BF588F00005A
:1013E000014B0360704700BF588F000010B5034BDE
:1013F0000360044606F030F9204610BD588F000007
:1014000010B5034B0360044606F026F9204610BDD4
:10141000588F000030B585B004AC04E90E00089C7C
:1014200034B94068194905B0BDE8304006F04CB900
:101430009DF80430022B07D0032B1DD11449627C88
:10144000406806F041F91BE0E268637C012A04D1A0
:10145000A26840680F4912780BE0022A07D1A16800
:1014600040680A784D780B4902EB052201E040689C
:10147000094906F029F903E00848094906F024F96A
:10148000204605B0BDE8304006F0C6BD888F00009C
:10149000B08F0000938F00009E8F0000E490FF1F2C
:1014A000B68F0000F8B5124F124B03600025FA26E4
:1014B000044680F87A5080F88E504160426680F889
:1014C000485080F86050C6662A463B4630460121A7
:1014D00003F07CF8C4F880602067012130462A467A
:1014E0003B4603F073F8C4F884002046F8BD00BF03
:1014F000E28F0000788F00004068014906F0E4B8F0
:10150000F28F00002DE9F041244BDFF894801B8816
:101510008AB005A9ADF81430D8F800301A680091E7
:101520000221002400F168070191D5698DF81D4062
:10153000184639460322FE23A8476D4607AE45F8F4
:10154000044B96E8070085E807002346D8F800001A
:101550003946224602F0C4FFD8F800008DF8194041
:101560001E238DF818308DF81A4006AA03680092E1
:1015700003220192D3F81CC03946FE23E0470094B1
:1015800096E8070085E807002346D8F800003946AA
:10159000224602F0A5FF0AB0BDE8F081688F000086
:1015A000BC88FF1F4068014906F08EB8819000009A
:1015B0000A4B10B5044618680023C21801330021F5
:1015C0000A2B82F88A10F8D1054B186802F0A8FDA2
:1015D00060680449FFF7C3FB10BD00BFB488FF1F5C
:1015E000BC88FF1FF89000002DE9F341674D684962
:1015F0000446406806F068F82868666801F01DFA3D
:1016000064490246304606F05FF82868666801F0D3
:101610001AFA61490246304606F056F828686668AC
:1016200001F017FA5D490246304606F04DF8286889
:10163000D4F8048001F016FA0746286801F018FA79
:101640000646286801F01AFA3346554900903A4692
:10165000404606F039F82868666801F01BFA5149DF
:101660000246304606F030F8286801F00DFA10B155
:1016700060684D4901E060684C4906F025F84C4926
:101680006068FFF75FFB2868666801F009FA49495E
:101690000246304606F018F82868676801F092F9AB
:1016A0000646286801F08BF932460346424938461F
:1016B00006F00AF82868676801F08AF90646286883
:1016C00001F099F9324603463C49384605F0FCFFE3
:1016D0002868666801F092F939490246304605F0FB
:1016E000F3FF2868666801F08CF9364B364A3749B3
:1016F000002818BF1A46304605F0E6FF34496068F6
:10170000224EFFF71FFB2868D4F8048001F086F909
:10171000074628682F4D01F07EF92F4903463A46C7
:10172000404605F0D1FF2868FFF75AFB38B32B4934
:101730006068FFF714FB3068D4F8048001F077F993
:101740000746306801F070F93A460346244940469E
:1017500005F0BAFF28686668FFF744FB2149024696
:10176000304605F0B1FF28686468FFF73DFB1E496D
:101770000246204602B0BDE8F04105F0A5BF606812
:101780001A49FFF7ECFA02B0BDE8F081B488FF1FF8
:101790003C91000059910000699100008491000083
:1017A00099910000B5910000D89100000F920000BF
:1017B000469200006E920000149300008792000091
:1017C000AD9200003591000039910000C6920000F2
:1017D000DF920000AC88FF1F0693000034930000E6
:1017E000639300008C930000A8930000C693000050
:1017F0002DE9F0416A4D2B680446D3F8AC0002F0A5
:10180000A5FE68490746606805F05EFF2B68D4F8BE
:101810000480986802F090FE0A2690FBF6F2624976
:10182000404605F051FF97FBF6F206FB12735F4945
:1018300060685F4F05F048FF2B685E49D3F8A4202D
:10184000606892FBF6F205F03FFF2B685A49D3F827
:101850009C206068594E05F037FF2B685849D3F833
:101860009820606805F030FF2B6856491A7B606845
:10187000002A0CBF3A46324605F026FF2B68524933
:101880001A69606805F020FF2B6850495A691B6986
:101890006068D21A05F018FF2B684D491A7E6068FF
:1018A000002A0CBF3A46324605F00EFF2B68494924
:1018B000DA69606805F008FF2B6847491A6A6068B2
:1018C00005F002FF4549606805F0FEFE444B4549BE
:1018D0001A78606805F0F8FE434B44491A7860684E
:1018E00005F0F2FE424B43491A78606805F0ECFEC1
:1018F0006068414905F0E8FE00262B68334493F800
:101900008A201AB160683D4905F0DEFE01360A2ED4
:10191000F3D160683A4905F0D7FE01262868676868
:10192000821992F87F1006F10B0250F8228049B11B
:1019300001F0B0F80146404602F00DFE3149034681
:10194000384608E001F0A6F80146404602F003FEE2
:101950002D49034638463246013605F0B5FE0B2EBA
:10196000DCD12A4D2868FFF73BFA90B1284960681E
:10197000FFF7F5F928686468FFF70EFA254B264A49
:101980002649002818BF1A462046BDE8F04105F058
:101990009BBE60682249FFF7E2F9BDE8F08100BF15
:1019A000B488FF1FFB9300000A94000029940000F4
:1019B000399100004A9400007494000035910000B1
:1019C00094940000B2940000D5940000FC940000B0
:1019D0002695000048950000699500008A95000052
:1019E0000091FF1FA6950000C388FF1FCC95000043
:1019F0000191FF1FF2950000179600007F920000F2
:101A0000389600004796000077960000AC88FF1FCC
:101A100096960000F4930000F7930000C59600002E
:101A2000C693000038B5184B45680446186801F0A5
:101A300010F816490246284605F046FE606814492B
:101A400005F042FE6068134905F03EFE60681249E9
:101A500005F03AFE6068114905F036FE60681049ED
:101A600005F032FE60680F4905F02EFE60680E49F1
:101A700005F02AFE60680D4905F026FE60680C49F5
:101A8000BDE8384005F020BEB488FF1FE196000095
:101A90000B970000DC970000EF970000FC97000018
:101AA00015980000379800006398000081980000A6
:101AB000A098000070B5294D46680446286800F0DB
:101AC000C8FF27490246304605F0FEFD60682549FB
:101AD00005F0FAFD6068244905F0F6FD60682349C9
:101AE00005F0F2FD6068224905F0EEFD60682149CD
:101AF00005F0EAFD6068204905F0E6FD1F496068D1
:101B000005F0E2FD2868666800F0C1FF1C49024646
:101B1000304605F0D9FD2868666800F0B8FF19491D
:101B20000246304605F0D0FD6068174905F0CCFD4F
:101B30006068164905F0C8FD6068154905F0C4FDE8
:101B40006068144905F0C0FD6068134905F0BCFDEC
:101B500060681249BDE8704005F0B6BDB488FF1F4B
:101B6000E1960000EE9800002D99000041990000D8
:101B7000689900008D990000C6990000D79900006F
:101B8000EA990000179A00005F9A0000A29A0000EC
:101B9000299B0000679B0000A49B0000D69B0000CF
:101BA0004068014905F090BD099C00002DE9F04F07
:101BB00003298BB00446894602D0FFF7F1FF61E0AC
:101BC000006D06F0E9F98246606D06F0E5F92F4BED
:101BD0005FFA8AFA83465146186800F069FF10B927
:101BE00060682B4904E0BBF5805F04DB606829492D
:101BF00005F06AFD46E0DFF8A480274BD8F8000026
:101C00001B88ADF8143005AA036800920222002553
:101C100004F168070192DC698DF81D5039464A4687
:101C20005346A0476C4607AE44F8045B96E80700AD
:101C300084E807002B46D8F8000039462A4602F00F
:101C40004FFC8DF819B0D8F800001E234FEA2B2B5B
:101C50008DF818308DF81AB006AA03688DE80402D2
:101C60003946D3F81CC04A465346E047009596E8EB
:101C7000070084E807002B46D8F8000039462A46BA
:101C800002F02EFC0BB0BDE8F08F00BFB488FF1F40
:101C90005A9C0000A69C0000688F0000BC88FF1FB3
:101CA0002DE9F041042988B0044602D0FFF778FFFF
:101CB00062E0006D06F070F90546606D06F06CF9A3
:101CC0008046A06D06F068F9FF2807464FDC2C4ED1
:101CD000EDB2306829465FFA88F800F0E9FE30B3CB
:101CE0008DF81170274F8DF81080386804A90023F3
:101CF0008DF8153003680091022104F16806019106
:101D000003228DF81420D3F81CC031462B46E0473F
:101D10006B4643F8044B08AC14E9070083E807005E
:101D20003146386801221E2302F0DAFB24E03068D5
:101D300000F0B6FE85421AD10A2384F868300323E6
:101D400084F86A3002236367236F84F8695083F84C
:101D50000080236F5F70306804F1680104F17C0239
:101D600001F0A2FB6068084994F88D2002E06068E9
:101D70000549082205F0A8FC08B0BDE8F08100BFC5
:101D8000B488FF1FBC88FF1FB08F00002DE9F04111
:101D9000032988B0044602D0FFF702FF61E0006D1E
:101DA000314E06F0F9F8C5B2606D06F0F5F8294637
:101DB000C7B2306800F07CFE50B3DFF8B8808DF811
:101DC0001070D8F80000012600238DF811608DF8FE
:101DD000153004A9022302688DF814308DE80A003A
:101DE00004F16807D2F81CC039461A462B46E04772
:101DF0006B4643F8044B08AC14E9070083E807007E
:101E00003946D8F8000032461E2302F069FB28E06C
:101E1000306800F045FE85421ED10A2384F8683000
:101E2000022384F86A306367236F84F869501F7057
:101E3000236F01225A70306804F1680104F17C02BA
:101E400001F010F9D4F8843060681A78074994F8E2
:101E50008D3005F039FC04E060680549082205F082
:101E600033FC08B0BDE8F081B488FF1F938F0000F9
:101E7000B08F0000BC88FF1F2DE9F041042988B015
:101E8000044602D0FFF78CFE62E0006D324F06F090
:101E900083F8C5B2606D06F07FF85FFA80F8A06D38
:101EA00006F07AF829460646386800F001FE40B38D
:101EB0002A4F8DF8116038688DF8108036128DF831
:101EC0001260032204A900238DF8153003688DF8F1
:101ED00014208DE8060004F16806D3F81CC03146D2
:101EE0002B46E0476B4643F8044B08AC14E9070067
:101EF00083E807003146386801221E2302F0F0FA19
:101F000026E0386800F0CCFD85421CD10A2384F815
:101F10006830032384F86A306367236F84F869505C
:101F200083F80080236F5E70236F36129E703868CE
:101F300004F1680104F17C0201F0B6FA6068084916
:101F400094F88D2002E060680549082205F0BCFB8A
:101F500008B0BDE8F08100BFB488FF1FBC88FF1F38
:101F6000B08F00002DE9F041032988B0044688466F
:101F700002D0FFF715FE5FE0006D314E06F00CF861
:101F8000C5B2606D06F008F82946C7B2306800F0A7
:101F90008FFD28B38DF810702A4F022238688DF813
:101FA000112004A900238DF8153003688DF8142042
:101FB0008DE8060004F16806D3F81CC031462B46B4
:101FC000E0476B4643F8044B08AC14E9070083E88C
:101FD00007003146386801221E2302F081FA2BE007
:101FE000306800F05DFD854221D1226F84F8695090
:101FF0000A2384F86830022384F86A30C4F87480B5
:102000001770226F5370306804F1680104F17C028C
:1020100001F028F8D4F8843060681A785B780A49AF
:1020200002EB032294F88D3005F04EFB04E060686B
:102030000649082205F048FB08B0BDE8F08100BF62
:10204000B488FF1FBC88FF1F938F0000B08F000073
:10205000022938B5044604D02046BDE83840FFF7D1
:102060009FBD056D0E49284606F0DDF840B90D4BC1
:10207000186800F0E1FF60680B49FEF770FE38BD9C
:1020800028460A4906F0CFF80028E5D1054C20681B
:1020900000F0B2FF2068BDE8384000F0DBBF00BFB1
:1020A0000E9D0000B488FF1F129D0000179D0000C8
:1020B000032970B504461AD1056D6B49284606F010
:1020C000B2F8C8B9656D6949284606F0ACF818B988
:1020D000674B0121186807E06649284606F0A3F817
:1020E000014620B9624B186800F08EFC71E0204672
:1020F000BDE87040FFF754BD28465F4906F093F8ED
:10210000A8B9656D5949284606F08DF818B9584B9D
:102110000121186808E05749284606F084F801466E
:102120000028E4D1524B186800F0D1FC51E0284659
:10213000524906F078F848B94D4B606D1D6805F0BE
:102140002BFFC1B2284600F06CFC42E028464C4907
:1021500006F069F8002841D1606D05F021FFCF2815
:10216000054602DD6068474935E0474B013093FB87
:10217000F0F005F0B1FC454905F0B6FD002106463A
:1021800005F0B0FE28B130464FF07C5105F0F0FB71
:1021900004E030464FF07C5105F0E8FB05F0B6FE58
:1021A0003B4A03464FF4165110685943FEF7E2FFCD
:1021B00010B16068374901E06068374905F084FA7A
:1021C0002B4BE9B2186800F035FC60683349FEF724
:1021D000C6FD60683249FEF7C2FD70BD2846314930
:1021E00006F021F870B92A4B616D1868FEF78CFF74
:1021F00010B160682C4901E060682C49BDE870406E
:1022000005F062BA28462A4906F00DF8C0B9606D9B
:1022100005F0C2FE42F20F739842014602DD60688B
:102220002449EBE71A4D2868FEF7D8FF0028E3D0D1
:1022300028686468FEF7D8FD1F49024620460FE073
:1022400028461E4905F0EFFF00287FF450AF104BE1
:10225000616D18686568FEF7F3FF19490246284664
:10226000BDE8704005F030BA1B9D0000279D0000BE
:10227000B488FF1F2B9D00002E9D00003E9D000096
:10228000469D00004D9D000080841E000000164603
:10229000AC88FF1F999D0000B89D0000D79D0000ED
:1022A000129D0000FB9D0000029E00000A9E00009F
:1022B000109E0000179E0000659E00009C9E00007E
:1022C000A69E0000022970B504460D4608D1006D97
:1022D0003C4905F0A8FF002849D102F09DFA6BE0C7
:1022E000032944D1056D3849284605F09CFF48B9BB
:1022F000364B606D1D6805F04FFE0146284600F024
:102300009FFB59E02846324905F08DFF48B92F4B15
:10231000606D1D6805F040FE0146284600F096FB02
:102320004AE028462B4905F07EFF48B9274B606DEF
:102330001D6805F031FE0146284600F0AEFB3BE08B
:102340002846254905F06FFFB0B9656D2349284639
:1023500005F069FF08B9282005E02846204905F066
:1023600062FF48B91E20012102F03CFA24E0206DF2
:102370001C4905F058FF20B12046BDE87040FFF72A
:102380000FBC052DF8D1114D606D2E6805F004FECF
:10239000C1B2304600F069FBA06D2E6805F0FCFD6F
:1023A000C1B2304600F067FBE06D2D6805F0F4FD2A
:1023B000C1B2284600F065FB60680B49FEF7CFFC10
:1023C00070BD00BFB19E0000B89E0000B488FF1F22
:1023D000C39E0000D19E0000E19E0000EC9E000024
:1023E000F19E0000F79E0000129D0000F8B5012349
:1023F0000B7090F848303F2B84BF03F1FF3380F817
:10240000483090F8482002440023137204460E46D8
:10241000012294F84800D9B288420CD92144097AA3
:10242000202905D12AB9327801323270012200E028
:1024300000220133EDE73378052BA8BF0523337065
:1024400004F10805002384F8603094F86070337854
:10245000BB421CD92846202194F8482005F0E4FD11
:1024600030B904EB87030137DD6484F86070ECE772
:10247000A84201D10135E8E704EB87070023FD649A
:10248000054605F8013B94F860300133DBE7E46C66
:102490003E49204605F0C7FE002859D020463C4959
:1024A00005F0C1FE002855D020463A4905F0BBFE94
:1024B000002851D02046384905F0B5FE00284DD0FF
:1024C0002046364905F0AFFE002849D02046344961
:1024D00005F0A9FE002845D02046324905F0A3FEAC
:1024E000002841D02046304905F09DFE00283DD00F
:1024F00020462E4905F097FE002839D020462C4969
:1025000005F091FE002835D020462A4905F08BFEC3
:10251000002831D02046284905F085FE00282DD01E
:102520002046264905F07FFE50B32046244905F099
:102530007AFE38B32046234905F075FE20B32046C5
:10254000214905F070FE002814BF01201120F8BDBC
:102550000220F8BD0320F8BD0420F8BD0520F8BD19
:102560000620F8BD0720F8BD0820F8BD0920F8BDF9
:102570000A20F8BD0B20F8BD0C20F8BD0D20F8BDD9
:102580000E20F8BD0F20F8BD1020F8BDFA9E000007
:10259000FF9E0000039F00000A9F0000109F0000A4
:1025A000229F0000189F00001E9F0000279F000030
:1025B0002E9F000013A00000CA9E0000369F00005E
:1025C0003A9F00003E9F0000429F000013B5044662
:1025D000606803689B689847002800F08480606802
:1025E0000368DB689847C0B20D28F1D00A2894F838
:1025F000483001D1012B01D83F2B6ED120460DF17F
:102600000701FFF7F3FE112860D8DFE800F06C093E
:102610000D1115191D2125292F353B41474D5359C2
:102620002046FFF7BDFA54E02046FFF743FA50E09A
:102630002046FFF7F7F94CE02046FFF7D9F848E0CD
:102640002046FEF7D1FF44E02046FEF7B1FF40E010
:102650002046FEF757FF3CE02046FEF7A3FF38E098
:1026600020469DF80710FEF747FF32E020469DF810
:102670000710FFF79BFA2CE020469DF80710FFF7A4
:10268000E7FC26E020469DF80710FFF71BFE20E040
:1026900020469DF80710FFF70BFD1AE020469DF835
:1026A0000710FFF7FDFA14E020469DF80710FFF72A
:1026B000E3FB0EE020469DF80710FFF767FB08E0FC
:1026C00020469DF80710FFF74DFC02E00D2001F0B9
:1026D00049FF002384F8483005E05A1C234484F85D
:1026E0004820187274E702B010BD10B5044600F01F
:1026F00027F8204610BDF0B589B06B4600248DF850
:10270000154043F8044B08AF06460D4617E907008D
:1027100083E80700304629462246234600F081F828
:1027200009B0F0BD08B500F0BEF8043008BD00F0F7
:10273000F5B800F0FFB800F0F4B800F0FDB8FFFF06
:10274000F8B504460D4616460846002228212A4BB5
:1027500001F03CFF294B2061012106FB05F000221E
:1027600001F034FF00236061DAB2AA4208D2226984
:10277000282101FB03220133D06096603044F3E747
:102780000C2101221E4B284601F020FF0C266FF081
:102790000B01034600F10C0216FB0511606006FBFD
:1027A000053682605A1820691860183E5A605660D3
:1027B000282606FB0506283E5E5093600122691E0E
:1027C0008A4213DA0C2112FB01F601FB023C9F192D
:1027D00011FB021119444CF8087CB96002EB82012C
:1027E00000EBC10101329951D2B2E8E7A360E36086
:1027F000002323702046F8BD469F00005F9F000025
:10280000839F000010B50446406905F005FC20696F
:1028100005F002FC606805F0FFFB002323702046F2
:1028200010BD2DE9F8439046027899460446836826
:1028300012B91D46E36009E0C568AA689A4205D14D
:10284000192001F08FFE0020BDE8F8832E68E368B0
:10285000B2689B68F068E3600F46331D01F1140E07
:1028600057F804CB43F804CB7745F9D1CB68B26075
:10287000F0609A42A8BF1A463261896802F08CF96A
:102880002968089A81F825902B6881F8248043F8FC
:10289000182B09AA07CA83E807002378013323709D
:1028A0000120BDE8F88310B5047814B18368186876
:1028B00010BD152001F056FE204610BD38B5037836
:1028C0008B4204460D4604DC1720BDE8384001F079
:1028D00049BE19B983689B6883601BE0013B99423C
:1028E00003D1C3685B68C36014E0182001F03AFEAE
:1028F000A368013D15F0FF059B68FAD15A689968F5
:10290000916099684A60E2689168996091685A603C
:102910004B6093602378013B237038BD0021FFF7A3
:10292000CDBF10B5044623781BB12046FFF7F6FF54
:10293000F9E710BD00787047C36880689A68131A79
:1029400058425841704710B580F8C23090F8C030F6
:1029500080F8C110044680F8C32090F8BD0093B100
:10296000C943C9B2013102F0C3FD94F8C31094F811
:10297000BE00C943C9B2013102F0BAFD94F8C210D9
:10298000C943C9B20BE0013102F0B2FD94F8C310A3
:1029900094F8BE00013102F0ABFD94F8C21094F837
:1029A000BF000131BDE8104002F0A2BD90F8C100A7
:1029B000704790F8C300704790F8C2007047D0F895
:1029C000C800704790F8C40070470B2001F0D6BED5
:1029D00090F8CC00704738B50546084685F8CC100D
:1029E0000C4601F0A7FD2146C5F8D0000C20BDE83B
:1029F000384001F0C3BED0F8D000704790F8D40042
:102A0000704790F8D60070470A461720012102B19E
:102A10000A4601F063BED0F8D800704790F8D7009E
:102A200070470F2001F0AABED0F8E000704790F880
:102A3000DC007047102001F0A1BED0F8E400704720
:102A4000002001F0B5BED0F8E8007047022001F088
:102A5000AFBE90F8F100704780F8F1100A201921FC
:102A600001F08CBE90F8F2007047042001F086BEA1
:102A700090F8F3007047052001F080BE90F8F40054
:102A80007047062001F07ABE90F8F0007047D0F849
:102A9000EC007047D0F8F80070471A2001F088BEAB
:102AA00090F8D500704780F8D5100E2001F066BE72
:102AB00059B10023C21892F88A208A4203D0013308
:102AC0000A2BF7D101E001207047002070470A4629
:102AD0001720002101F002BE90F8F51010B5044651
:102AE000B1B9D0F8E43090F8A100032B02D102F084
:102AF000E3FC07E0012102F0DFFC94F8A1000121D2
:102B000002F0BAFC322002F0F5FD012384F8F53022
:102B100010BDFFFF2DE9F04104460A2001F0D2FD6F
:102B2000192884F8F10003D020461921FFF794FFFB
:102B3000002001F0CDFDC4F8E400022001F0C8FD42
:102B4000C4F8E8000D2001F0BDFD84F8D4000C208D
:102B500001F0B8FD84F8CC0001F0ECFCC4F8D00022
:102B60000B2001F0AFFD84F8C40001F0C9FC012185
:102B7000C4F8C800172001F093FD003018BF0120F1
:102B800084F8D6000E2001F09DFD84F8D5000F20BA
:102B900001F098FD84F8D70001F0B2FCC4F8D80029
:102BA000102001F08FFD84F8DC0001F0A9FCC4F8CE
:102BB000E000042001F086FD84F8F200052001F019
:102BC00081FD84F8F300062001F07CFD002184F8EB
:102BD000F40084F8BC10172001F062FD003018BF2B
:102BE000012084F8F00010B140F6FF7301E040F2DC
:102BF000FF33C4F8EC30D4F8E83003F0010222735C
:102C0000C3F3400222765A0701D5322304E01B07A2
:102C10004CBF4A234FF0FF330025C4F8A43084F89A
:102C2000F5501A2001F054FDD4F8E830C4F8F8004B
:102C300013F0160F0CBF0023012384F8C0304FF4AB
:102C40004873C4F8B0304FF49663C4F8B43001212F
:102C500040F2DC53C4F8B8300A200A46D64B01F0E3
:102C6000B5FCD4F8E4702060032F79D102234FF033
:102C7000040884F8A0304046012184F8BD8002F0A9
:102C80001BFC052084F8BE00012102F015FC062083
:102C900084F8BF00012102F00FFC2A46772320466A
:102CA0003321FFF750FE12200121607302F004FC73
:102CB0002520A07302F02CF919236061637620614E
:102CC0000F230B20A376012184F8A200242602F012
:102CD000F3FB1D2084F8A860207102F019F9A060B0
:102CE00094F8A80002F014F91A2384F824301C2365
:102CF00084F82530152384F82630102384F82730F3
:102D00001F2384F8A130C4F8AC002946092084F8B8
:102D1000286084F8296084F82A6084F82B6084F89D
:102D20002C6084F82D6084F8946084F8956002F03B
:102D3000C3FB2020294602F0BFFB3846294602F09B
:102D4000BBFB0C20012102F0B7FB9C4B80221A60D8
:102D50001320012102F0B0FB994BC3F800800AE177
:102D6000042F70D1022384F8A030384684F8BD7057
:102D7000012102F0A1FB052084F8BE00012102F030
:102D80009BFB062084F8BF00012102F095FBFF2287
:102D90002B4620462946FFF7D6FD1E2060730121F1
:102DA00002F08AFB1D20A07302F0B2F819236061C3
:102DB00063762061212320200121A37684F8A200DC
:102DC00002F07AFB1F230F2084F8A830207102F054
:102DD0009FF8A06094F8A80002F09AF81C2384F8E9
:102DE00024301B2384F82530242384F8263025231F
:102DF00084F82730112384F82830132384F82930ED
:102E0000142384F82A30152384F82B30172384F8F0
:102E10002C30162384F82D30122384F894301A2392
:102E2000C4F8AC0084F895301020012102F044FB76
:102E30002946102002F020FB0E2084F8A100012179
:102E400002F03AFB97E0052F40F091800223152015
:102E500084F8A03084F8BD00012102F02DFB384633
:102E600084F8BE70012102F027FB062084F8BF0021
:102E7000012102F021FBFF222B4620462946FFF7C5
:102E800062FD14206073012102F016FB1020A07374
:102E900002F03EF81923606163762061212320202F
:102EA0000121A37684F8A20002F006FB1F230F2065
:102EB00084F8A830207102F02BF8A06094F8A800E4
:102EC00002F026F81C2384F824301B2384F82530D4
:102ED000242384F82630252384F82730112384F80E
:102EE0002830132384F82930232384F82A3022231E
:102EF00084F82B30172384F82C30162384F82D30D7
:102F00001223C4F8AC0084F894300E201A2384F8FD
:102F1000953084F8A100012102F0CEFA09200121A8
:102F200002F0CAFA2946092002F0A6FA0B20012174
:102F300002F0C2FA29460B2002F09EFA0C20012171
:102F400002F0BAFA29460C2002F096FA1D2001215F
:102F500002F0B2FA29461D2002F08EFA1E2001214D
:102F600002F0AAFA1E20294602F086FA03E0FE23A8
:102F7000C4F8E4303CE02046FFF7AEFD207901F0D4
:102F8000C7FF237EA06043B1607E03F037FCE061A1
:102F9000A07E03F033FC206201E0E3612362237B27
:102FA00083B1607B012102F087FAA07B01F0B0FFC2
:102FB0002061236907E000BF05A0000088F00F40F2
:102FC00048F00F402361636104F10A06254600239F
:102FD00085F88A30A36595F8240085F880302F1B8A
:102FE00001F096FF0C370135B54244F82700EED1C9
:102FF0002046BDE8F08100BF10B5D0F8E430032BC7
:10300000044690F8A1000ED1012102F055FA94F87F
:10301000A120084B53F83230012283F8802064202D
:1030200002F068FB02E0002102F026FA002384F897
:10303000F53010BDC4AD000010B50446FFF7DCFF4D
:103040004FF4967002F056FB2046BDE81040FFF7A3
:1030500043BDFFFF014B024A1A6070470CED00E0D0
:103060000400FA052DE9F74F8B68914693F800A00C
:103070005A78D9F804300AF1FF3B9A42B8BF134698
:103080009B444FF00008DBB2C9F80C3089F811807E
:103090000446FFF7FFFC5FFA8BFB07460AEB0803C9
:1030A000DBB25B4500F2F3815FFA88F5D9F808607E
:1030B000B82B00F2E781DFE813F0B9001301BB0081
:1030C000BF00C300E501E501E501E501E501E5011A
:1030D000E501E501E501E501E501C700E501E501DF
:1030E000E501CB00E501E501E501E501E501E501CB
:1030F000E501E501E501E501E501E501E501E501A0
:10310000E501E501E501E501E501E501E501CF00A6
:10311000D400E501E501E501E501E501E501E50191
:10312000E501E501E501E501E501E501E501E5016F
:10313000E501DB00E501DF00E300E700EB00EF0065
:10314000F300F6000401E50109011301E5010D0199
:10315000E5010F011301E5011501E50117011D014D
:10316000E5011B01E5011D0133011F0124012901B6
:103170002E01E50138013A014301E5014C014E0100
:10318000530158015D01E501620168016E01790199
:10319000E5018501870189018B018D018F01910175
:1031A00093019501970199019B019D019F01A10147
:1031B000A301A501A701A901AE01E501B501B8016F
:1031C000BB01BE01C101C401C701CA01CD01D001CB
:1031D000E501E501E501E501E501E501E501E501BF
:1031E000E501E501E501E501E501E501E501E501AF
:1031F000E501E501E501E501E501E501E501E5019F
:10320000E501E501E501E501E501E501E501E5018E
:10321000E501E501E501D301E501D601E501D901AB
:10322000E501DC01E501DF01E501E20195232AE189
:103230002046FFF70EFCF3E02046FFF731FCEFE0FD
:103240002046FFF7BFFBEBE02046FFF7D7FBE7E0A8
:103250002046FFF719FCE3E0D4F8AC0001F076F962
:10326000DEE0A06801F068F90A2390FBF3F0D7E0F4
:103270002046FFF7E2FBD3E02046FFF7E4FBCFE078
:103280002046FFF7E0FBCAE02046FFF7EBFBC7E074
:103290002046FFF7EDFBC3E02046FFF7EFFBBFE062
:1032A00094F8F530EFE02046FFF783FB0346204615
:1032B0000193FFF77BFB019B23F00F0303EB20102F
:1032C000AEE02046FFF778FB0011A9E02046FFF7AB
:1032D00098FBA5E06F4BC4E02046FFF79FFB9FE003
:1032E0000123D0E06C4BBCE02046FFF7A0FB97E049
:1032F0006A4BB6E00323C6E0694B1868FDF770FD22
:103300008EE0674B1868FDF747FD89E0644B18684D
:10331000FDF76AFD84E0624B1868FDF765FD7EE00D
:10332000604B1B6893F8BC30ADE0237BABE02046DC
:10333000FFF7AAFB62692369D31A23EAE3732FE03C
:103340002046FFF7A1FB62692369D31A23EAE373DE
:1033500031E0237E97E02046FFF796FBE3691FE00C
:103360002046FFF791FBE36925E02046FFF78CFB41
:10337000236A15E02046FFF787FB236A1BE02046FF
:10338000FFF782FBD4F89C300AE02046FFF77CFB75
:10339000D4F89C300FE02046FFF776FBD4F8983045
:1033A00008B1DBB26FE0C3F387036CE02046FFF7A0
:1033B0006BFBD4F8983010B1C3F3072363E0C3F379
:1033C000872360E0206B22E0206B25E0606B1EE02D
:1033D000606B21E0A06B1AE0A06B1DE0E06B16E0D3
:1033E000E06B19E0206C12E0206C15E0606C0EE0E0
:1033F000606C11E0A06C0AE0A06C0DE0E06C06E0EF
:10340000E06C09E0206D02E0206D05E0606D39465A
:1034100001F0A1F804E0606D394601F09CF800125B
:10342000705531E094F88A302DE094F88B302AE022
:1034300094F88C3027E094F88D3024E094F88E30A6
:1034400021E094F88F301EE094F890301BE094F85F
:10345000913018E094F8923015E094F8933012E02F
:1034600023681B780FE023685B780CE023689B7867
:1034700009E02368DB7806E023681B7903E0236812
:103480005B7900E00023735508F1010806E603B0FC
:10349000BDE8F08F0091FF1FC388FF1F0191FF1F40
:1034A000AC88FF1FB488FF1F2DE9F74F8B680027FA
:1034B000D760577493F800A0CB680AEB030BABF10D
:1034C000020B0546894616465FFA8BFBB846FAB2F0
:1034D00002EB0A03DBB201325B45D2B200F2158186
:1034E000D9F80810822B8C5C00F0E8803FD8442B80
:1034F00000F09A8015D8052B00F0058109D8032B20
:103500006BD0042B40F0FB8028462146FFF75DFA84
:10351000F9E0142B75D0432B7BD0102B40F0EF80BB
:1035200067E05A2B00F09A8019D8572B00F0AA8038
:10353000592B00F08A80452B40F0E1802846FFF7A8
:1035400035FA014628460191FFF733FA04F00F04DB
:1035500004EB0413024601992846DBB272E0802B8B
:1035600000F0A38000F2A7805B2B79D0C7E0892B05
:1035700000F0B38015D8852B00F0A68009D8832BE6
:1035800000F09F80842B08BF85F88D4000F0BB8041
:10359000B5E0872B00F09B8000F29C8085F88F407F
:1035A000B1E0B22B00F0A2800BD8AE2B00F09880D7
:1035B000B02B00F098808A2B40F0A18085F89340D2
:1035C000A1E0B62B00F09580B82B00F09580B42BCD
:1035D00040F095802B68DC7095E028462146FFF787
:1035E00067FA002840F08B8028462146FFF75BFAF7
:1035F00089E0022C00F2838028462146FFF7EBF990
:1036000081E028460CB9214600E00021FFF75FFA6F
:1036100079E01CB92846FFF7EFFC74E0012C6ED16D
:103620002846FFF759FA6EE02846FFF7C5F904F07F
:103630000F01241101EB011104EB04120346C9B27E
:103640002846D2B2FFF77FF95DE0314B186814B914
:10365000FDF7B2FB57E0FDF7A1FB54E0A04652E0B6
:1036600008EB042142F20F73994204DC284B1868DE
:10367000FDF7B4FD03E0737C43F0080373744FF06F
:10368000000840E014F0E00239D123462BB1D907FD
:1036900044BF0132D2B25B08F8E7022A00D074BB03
:1036A0001C4B1B6883F8BC402DE064B31A4B1868B0
:1036B00000F036FD27E085F88A4024E085F88B404D
:1036C00021E085F88C401EE085F88E401BE085F8EF
:1036D000904018E085F8914015E085F8924012E09E
:1036E0002B681C700FE02B685C700CE02B689C70E2
:1036F00009E02B681C7106E02B685C7103E0737CA9
:1037000043F0080373740137E1E603B0BDE8F08FBE
:10371000AC88FF1FB488FF1FBC88FF1F38B5856ABF
:10372000084B036004462DB12846FFF76BF8284686
:1037300003F092FF201DFDF7CFFD034B23602046D1
:1037400038BD00BF20A00000588F000010B504460F
:10375000FFF7E4FF204603F07FFF204610BDFFFF88
:103760002DE9F04106461C4B46F8043B0446002573
:10377000904630460F46FDF787FD3046414684F8B7
:103780002C5084F8425084F856502577FDF79AFD66
:10379000A761124FFA2666632A463B46304601214E
:1037A00000F014FF3B462A46A063A6640121304680
:1037B00000F00CFFE064182003F04CFF0F21022200
:1037C0000646FEF792FF0123A66284F82C50237769
:1037D0002046BDE8F08100BF20A00000E28F00007D
:1037E00038B50446806903689B689847E8B1251D91
:1037F0002846FDF7D5FDA06903689B68984718B176
:103800002846FDF7A9FD38B194F82C301BB1074BC1
:103810001B68636238BD38BDA0690368DB689847E0
:10382000C1B22846FDF762FDE5E738BD0089FF1FFC
:1038300082B030B585B00C4608A981E80C006B4613
:1038400043F8040B07C983E80700064B9DF82C20BA
:10385000186821461E2300F043FE05B0BDE8304045
:1038600002B07047BC88FF1F10B586B000240193DA
:10387000059B00938DF80D408DF80C2003AB0CCB0D
:10388000FFF7D6FF06B010BD10B50446806AFEF7FC
:1038900052FF002384F82C3010BD38B54C78CB682B
:1038A00002341C440B780A2B0D46E4B201D18B780C
:1038B00002E0142B03D14B7C1C44E4B202E00E2046
:1038C00000F050FEE96800238B4205DAAA68D25C5A
:1038D0001444E4B20133F7E7E043C0B238BD8329B2
:1038E00006D003D80139022904D801E0922901D178
:1038F000012070470020704738B50446806903688E
:103900000D461B68FF219847A0690368FF211B68CB
:103910009847A069697803681B689847A069E968B7
:10392000036802311B68C9B29847A069697C0368C3
:103930001B689847A069A9680368EA685B689847AC
:10394000A069297C03681B68984738BD70B51423AB
:1039500080F844308B780022013B04460D4680F805
:103960005520052B26D8DFE803F003081325251E74
:103970006B7880F8453002651CE06B7880F8453044
:103980001F4B2946186804F14402FFF76BFB11E056
:103990006B7880F845301A4B2946186804F14402C8
:1039A000FFF782FD06E0164E3068FFF725FB306812
:1039B000FFF750FB94F84530FE2B1FD0AB7CEBB9E2
:1039C0000F4E3068FFF71AF8022809D03068FFF769
:1039D00015F80128AB7801D1022B01D0012B0DD1B4
:1039E00004F1440529462046FFF757FF84F85400A8
:1039F00029462046BDE87040FFF77EBF70BD00BF7E
:103A0000B488FF1F2DE9F04F8B6885B01A7893F8C2
:103A100001B0039207460D460224EB689C4246DA49
:103A2000DFF89480AB68D8F800001E5DFFF738F827
:103A300086420BF1010A05D0D8F800003146FFF7A5
:103A400037F800B3AB68039A1A551A4B1868AB687D
:103A50000268234400935FFA8AF3019307F1440953
:103A6000D2F81CC0494603223346E047D8F800008C
:103A7000FFF716F8864209D1012387F856303846F9
:103A80004946FFF763FF5444E4B2C6E70A4B3146A8
:103A90001868FFF70DF830B1384649460222012375
:103AA000FFF7E2FEEFE7122000F05CFDEBE705B068
:103AB000BDE8F08FBC88FF1FB488FF1FF8B504462F
:103AC000A06AFEF736FE002804DC2046BDE8F84078
:103AD000FFF7DABEA06A174FFEF724FE45780646C8
:103AE0003868FEF7DDFF85423146204602D1FFF7F8
:103AF0002DFF03E003220123FFF7B6FEA06AFEF7C5
:103B000016FE0D4B38681B686362FEF7C9FF8542DD
:103B10000FD1A06AFEF70DFE002806DDA06AFEF7B1
:103B200001FEC37CAB42CBD0F8BD94F82130AB4250
:103B3000CBD0F8BDB488FF1F0089FF1F38B5012323
:103B400080F82C30084B90F820501B6843620446E4
:103B5000806AFEF7E7FD4378AB4204D12046BDE81A
:103B60003840FFF7ABBF38BD0089FF1F2DE9FF4785
:103B70008B68876C9B7880F820308A68CB68C66C2D
:103B80001344044613F8023C80F8213000F1440845
:103B90003A4630460D46002104F070FA40460021B6
:103BA000142204F06BFA4FF0FF09E664A7640126C3
:103BB000EB689E4238DA771CDFF87CA0AB68DAF855
:103BC0000000D95DFEF774FF38B9DAF80000FEF79F
:103BD00067FFAB68DB5D834220D1A06AFEF7ADFDD5
:103BE00010B11A2000F0BEFCAB689A1992788DF8DB
:103BF0000C209A5D8DF80D200E4ADB5D106803AA3B
:103C00000168009202220192D1F81CC04146E047AF
:103C100084F85790A06A4146FEF76DFDAB68033605
:103C200013F80790F6B2C3E72046FFF787FF04B00A
:103C3000BDE8F087BC88FF1FB488FF1F037F2DE914
:103C4000F0470446002B00F0DF8090F82C302BB1B9
:103C50006E4B1A68436AD31A642B19D82046FFF7B3
:103C6000BFFD251D2846FDF757FB05280EDD28461C
:103C70000021FDF75BFBFF2840F0C18028460121B1
:103C8000FDF754FBFF2840F0BA8004E0BDE8F08760
:103C9000FFF7FAFDE2E702212846FDF747FB002384
:103CA00084F8310084F8423028460321FDF73EFBBA
:103CB0000128074607DD2846FDF72EFBFB1C834243
:103CC00003DBBDE8F087BDE8F08794F82C304BB1FA
:103CD000142384F8303028460421FDF727FB84F8AC
:103CE000410008E00A2384F8303028460421FDF71B
:103CF0001DFB84F83200626BBB1E9342A8BF1346C3
:103D000003F10508E3635FFA88F80526F3B243453B
:103D10000BD231462846D4F83890FDF707FBA6F1C0
:103D2000050A013609F80A00F0E741462846FDF782
:103D3000FDFA04F1300684F8400031462046FFF7D2
:103D4000ACFD94F84030834259D194F82C3083B1C3
:103D5000A06AFEF7EEFC002845DDA06AFEF7E2FC53
:103D600094F83130C27C9A423DD12046FFF7A6FE3E
:103D700042E0204694F83210FFF7B1FD00283BD016
:103D8000DFF88C8094F83190D8F80000FEF788FEB8
:103D9000814523D0D8F8000094F83110FEF788FE52
:103DA000034630B10122204631461346FFF75CFD41
:103DB00022E094F83120FE2A1ED194F83220832A82
:103DC0002046314602D1FFF71DFE15E0922A02D1AE
:103DD000FFF7CCFE10E00222FFF746FD20463146F9
:103DE000FFF7B4FD08E094F8212094F831309A42AE
:103DF00002D12046FFF748FD2846391D01E028463C
:103E00000121FDF7B7FA2CE7BDE8F0870089FF1F15
:103E1000B488FF1F30B585B004AD05E90E00089DDC
:103E20009DF804300446002D34D0012B05D12946DD
:103E300005B0BDE83040FFF75FBD032B22D190F8FD
:103E40002C30A3B12946FFF757FD134BA06A1B681E
:103E50006362FEF76EFC002809DDA06AFEF762FCD3
:103E60006B78C27C9A4202D12046FFF727FE6A781F
:103E700094F821309A420DD1204605B0BDE830407B
:103E8000FFF702BD022B05D0132005B0BDE830407E
:103E900000F068BB05B030BD0089FF1F38B5056D67
:103EA000074B036004462DB12846FDF715FA284656
:103EB00003F0D2FB204600F0E3FA204638BD00BFF5
:103EC00038A0000010B50446FFF7E8FF204603F0D5
:103ED000C3FB204610BD2DE9F04186B004688DF883
:103EE00014209846022205AB8E4600F13C07009351
:103EF00001920126734639468DF81560E46905463E
:103F0000A0476C460CAB44F8048B93E807001E23D3
:103F100084E8070028463946324600F0E1FA06B048
:103F2000BDE8F081F0B587B000F13C058DF81530A3
:103F300005AB8DF8142002680093022301930F460D
:103F4000D66929463B4603220446B0476B460C9A85
:103F500043F8042B0DAA07CA83E807002046294628
:103F60009DF840209DF8443000F0BAFA07B0F0BD4B
:103F7000F0B587B004688DF814201F46022205AB07
:103F80008E4600F13C060093019273468DF8152091
:103F90003146E4690546A0476C460CAB44F8047B07
:103FA00093E807001E2384E80700284631460122D3
:103FB00000F096FA07B0F0BDF0B587B006688DF84E
:103FC00015301B128DF814208DF81630032205AB26
:103FD00000F13C05009301920F463B462946F669E5
:103FE0000446B0476B460C9A43F8042B0DAA07CA47
:103FF00083E80700204629469DF840209DF844307C
:1040000000F06EFA07B0F0BD2DE9F04188B005ACC4
:1040100084E80E009DF814200E9B9DF816509DF824
:104020001780012A064632D14BB1092D35D81C49DB
:104030005B7809686A1C0D4485F88A30D5B2B8F1FE
:10404000FC0F2AD8092D28D83268002308F101086E
:10405000009301935FFA88F806F13C07D2F81CC080
:104060003046394643460122E0476B468DF81650EC
:104070008DF8178043F8046B94E8070083E8070085
:10408000304639460122062300F02AFA05E00420D2
:1040900008B0BDE8F04100F065BA08B0BDE8F081B5
:1040A000B488FF1F10B5002241600446034B084648
:1040B000012100F08BFAA06010BD00BFE28F00006C
:1040C000F8B5044617460E46002500F0F7F9134BE5
:1040D0002360666584F8265084F83A5084F84E5080
:1040E000142003F0B7FA0646FDF7CEF830463946FD
:1040F0002665FDF7E7F804F11400FA21FFF7D2FF77
:1041000004F12800FA21FFF7CDFF04F13C00FA2169
:10411000FFF7C8FF25712046F8BD00BF38A000009A
:10412000F0B5184B0546186889B000228118013295
:1041300000230A2A81F88A30F8D12A6800930124E2
:10414000019305F13C068DF815308DF81630D769CE
:104150008DF814402846314622462346B8476B4620
:104160008DF8174043F8045B08AF17E9070083E8B0
:104170000700284631462246062300F0B1F909B06F
:10418000F0BD00BFB488FF1FF0B589B004AA0523B5
:104190008DF81030036800920222002400F13C06E2
:1041A0000192DF698DF8154031468DF811400322E8
:1041B000FE230546B8476B4608AF43F8044B17E9A2
:1041C000070083E80700284631462246234600F0D0
:1041D00087F909B0F0BD38B54C78CB6802341C447F
:1041E0000B780A2B0D46E4B201D18B7802E0142B38
:1041F00003D14B7C1C44E4B202E00B2000F0B2F986
:10420000E96800238B4205DAAA68D25C1444E4B260
:104210000133F7E7E043C0B238BD2DE9F0474E68FF
:104220008D68089F0C4691460021324680462846FC
:104230009A4603F023FF14222046002103F01EFFBC
:104240009DF8242066600A23B242A8BF3246A560CA
:10425000237084F801A084F80290E2601FB1284620
:10426000394600F099FC40462146FFF7B4FF207420
:10427000BDE8F0872DE9F8430446006DFDF74CF8E2
:10428000012827DD206D0021FDF750F8FF2805D11A
:10429000206D0121FDF74AF8FF2804D0206D01218F
:1042A000FDF768F816E0206DFDF736F8052811DDFA
:1042B0000221206DFDF73AF803210546206DFDF738
:1042C00035F80128064605D9206DFDF725F8F31CC1
:1042D000834201DB002533E0142365752375206DCF
:1042E0000421FDF723F8A36984F82500B71E9F4237
:1042F000A8BF1F4627620537FFB20525EBB2BB42B8
:104300000BD22946206DD4F81C80FDF70FF8A5F1DB
:104310000509013508F80900F0E73946206DFDF779
:1043200005F804F11405074684F8240029462046C0
:10433000FFF751FF8742206DB1D1311DFDF71AF80B
:104340002846BDE8F88338B50546406D0A230B7052
:1043500003680C461B68FF219847686D0368FF21BE
:104360001B689847686D617803681B689847686D9B
:10437000E168036802311B68C9B29847686DA1788B
:1043800003681B689847686DA1680368E2685B680A
:104390009847686D217C03681B68984738BDFFFF0C
:1043A000F7B50446606D03689B68984758B1606D27
:1043B0000368DB689847C1B2206DFCF797FF2F4B6D
:1043C0001B68A360EEE726792EBBE068FEF7B2FA21
:1043D000002851DD206DFCF7C9FFE068FEF763FAA5
:1043E00046760546061D31462046FFF7ACFF6B7941
:1043F000FE2B06D1062001F07DF920463146FFF75D
:10440000A2FF95F82430237113B9E068FEF786FA0D
:104410001A4B1B6819E0012E19D1E068174FFEF7FF
:1044200042FA05462046FFF725FF3A68A368A0B97F
:1044300095F82510D31A8B421ED96B7E6BB96E7618
:104440002046291DFFF77FFF3B68A36014E00C2086
:1044500003B0BDE8F04000F085B82B683BB11A68A6
:10446000009018351668184695E80E00B047E068C9
:10447000FEF754FA0023237103B0F0BD0089FF1F3B
:1044800038B5C568064B036004462DB12846FEF7D3
:10449000B9F9284603F0E0F8024B2360204638BD06
:1044A00068A00000588F000010B50446FFF7E8FF31
:1044B000204603F0D1F8204610BDFFFF38B5074B6A
:1044C00003600446182003F0C5F80F210546FA22C0
:1044D000FEF736F9E560204638BD00BF68A0000051
:1044E000F0B505AC1646059A44F8042B05460F4670
:1044F000E86839463246BDE8F040FEF792B9FFFF62
:10450000FB280CD0FC2803D0FA2803D105487047BB
:1045100005487047054B0130B3FBF0F07047044885
:10452000704700BF10552200C0C62D0080841E00B9
:10453000A0252600400070478010EE38024B20EA8C
:10454000E07053F82000704790A0000040F26B1319
:104550005843000B704740F2DE735843B0FBF1F054
:104560007047FFFF70B505462C46002C23DD012D5A
:1045700012DD134E306878B100221346FF21FEF79A
:10458000E2F94FF47A7001F0B5F8002130680A467C
:104590000B46FEF7D8F908E00A4B20261E604FF4C0
:1045A0007A7001F0A7F8084B1E604FF47A7001F0A2
:1045B000A1F8013CD9E74FF47A6001F09BF8D3E70A
:1045C000B488FF1F84F00F4088F00F4070B51E467E
:1045D00001FB00F412B103F0E7FC02E0204603F017
:1045E00013FD0C490B6803B908600B4D0B6808609C
:1045F000C21A2B6813442B60084D2B681C442C6096
:1046000038B907480749324603F05EF81420FFF72F
:10461000A9FF70BDC888FF1FC488FF1FCC88FF1F7B
:10462000E490FF1FA0AC0000054B1A6840F6B733BA
:104630009A42014602D9034803F010B8704700BF00
:104640000089FF1FE490FF1F08B5084B1A6840F669
:10465000B7339A42014607D9054802F0FFFF0448E4
:10466000BDE8084003F01AB808BD00BF0089FF1F6D
:10467000E490FF1F08B5084B1A6840F6B7339A421A
:10468000014607D9054803F064F80448BDE808402E
:1046900003F004B808BD00BF0089FF1FE490FF1FAE
:1046A000072910B50C460BD872B600F08BFD62B628
:1046B0000123A3401840C0B240FA04F4E0B210BD98
:1046C000002010BD08B572B600F07CFD62B608BDD2
:1046D00008B572B600F08AFD62B608BD2DE9FF414B
:1046E000234D2B68642B07460C4690462E460DDD65
:1046F0002049684603F094F86846FFF795FF68463E
:1047000003F04EF82868FFF7B5FF2DE0072921D800
:1047100000F080FD0028FBD072B6384600F052FD54
:1047200062B6012303FA04F418F0010F0CBF20EA6B
:1047300004040443E4B200F06DFD0028FBD072B61F
:104740003846214600F06EFD62B6336801333360AF
:1047500001200AE00849684603F062F86846FFF75E
:1047600073FF684603F01CF8002004B0BDE8F08138
:10477000D088FF1FCCAC000021AD000070B50B4C01
:104780002368642B05460E460EDC00F043FD00282E
:10479000FBD072B62846314600F044FD62B623686D
:1047A00001332360012070BD002070BDD088FF1F41
:1047B00070B50B4C2368642B05460E460EDC00F0EA
:1047C00029FD0028FBD072B62846B1B200F044FDA6
:1047D00062B6236802332360012070BD002070BDE3
:1047E000D088FF1F10B5044659B101210B20FFF7F7
:1047F000C5FF00210C20FFF7C1FF0D200221FFF7AC
:10480000BDFF631EDBB2FC2B05D821460E20BDE8A0
:104810001040FFF7B3BF10BD08B500210220FFF71D
:10482000C7FF00211720FFF7C3FF00210122172037
:10483000FFF754FF01210A461720FFF74FFF41F20F
:1048400044611A20FFF7B4FF03210F20FFF796FF02
:1048500010200146FFF792FF01211320FFF78EFF82
:1048600001211420FFF78AFF03211520FFF786FF9F
:1048700003211620FFF782FF01200146BDE8084012
:10488000FFF7B0BF084B1A6842F480721A604FF409
:10489000A072013A7FF4FDAF1A689205FCD4202380
:1048A000013B7FF4FDAF7047005004402DE9F74F06
:1048B0006A4E6B4B3268517E927E5C5C9D5CFF2C35
:1048C000814601D0FF2D02D11120FFF74BFE316848
:1048D000644A4B7E644F02EBC303586800230360B5
:1048E000897E624802EBC102614952681360614BE4
:1048F000620013440B605F4B6A0013443B605E4BE5
:104900001A6842F020021A6001235C4A03FA05F596
:1049100003FA04F445EA04031360594B1A6822F0C1
:1049200080021A60574A1060574818608846B9F1EB
:10493000000F7AD0142000F0DDFEFFF7A3FFD8F8B7
:10494000003052491B889BB2ADF80030BDF80030F2
:10495000BDF800204E4B92B20A601A603A684D4989
:10496000128892B2ADF80220BDF80220BDF80220F4
:1049700092B20A6048494FF00A0A0A609946FFF766
:1049800081FFD8F80030414D1B88D9F800203868E5
:10499000404C9BB2ADF80430BDF80430BDF80410B3
:1049A0003E4B89B219602B684FF0060B42F20F7E26
:1049B0000BFB02120EFB031342F21071B3FBF1F377
:1049C0002B6003889BB24FF0070CADF80630B2FBAA
:1049D000FCF2BDF80630BDF80600C9F800202268D8
:1049E0002F4B80B20BFB0202DFF8ACB01860DBF893
:1049F00000300EFB0303B2FBFCF2B3FBF1F1052028
:104A00000AF1FF3A2260CBF8001000F073FE1AF0B2
:104A1000FF0AB4D11E4A336811682A688A1ADA611B
:104A20002168DBF800208A1A1A62154B15491A68AA
:104A300022F080021A600A6842F420620A601A6852
:104A400042F0D2021A60174B80221A70A3F24B3345
:104A50004FF400221A6003B0BDE8F08FB488FF1F46
:104A600078AD0000C4AD0000F088FF1F0000030314
:104A7000EC88FF1F00510440388004400850044077
:104A8000005004400450044080004D00F488FF1F93
:104A9000E888FF1FE088FF1FD488FF1FE488FF1FFE
:104AA000DC88FF1F53E400E02C4BF7B51A6812F4C2
:104AB000805F1A680AD042F480521A60284B1A6844
:104AC000002001321A60FFF7F1FE45E042F4004297
:104AD0001A60244B1B681B889BB2ADF80430BDF8EC
:104AE0000430BDF80420204B92B21A601F4B1C68A2
:104AF0004FF0060C07270CFB0424B4FBF7F41C60F2
:104B00001B4B196842F20F7606FB012242F2107528
:104B1000B2FBF5F21A60174B17491B681B889BB252
:104B2000ADF80630BDF80630BDF806309BB20B601C
:104B3000124908680CFB0030B0FBF7F00860104920
:104B40000F6806FB0733B3FBF5F30B600D490968EB
:104B5000A21AC31ACA610B6203B0F0BD0050044030
:104B6000D888FF1FEC88FF1FE488FF1FE888FF1F1D
:104B7000F488FF1FF088FF1FDC88FF1FE088FF1FFD
:104B8000D488FF1FB488FF1F024B4FF400221A6025
:104B9000704700BF88E100E0844641EA000313F05B
:104BA00003036DD1403A41D351F8043B40F8043B34
:104BB00051F8043B40F8043B51F8043B40F8043BF7
:104BC00051F8043B40F8043B51F8043B40F8043BE7
:104BD00051F8043B40F8043B51F8043B40F8043BD7
:104BE00051F8043B40F8043B51F8043B40F8043BC7
:104BF00051F8043B40F8043B51F8043B40F8043BB7
:104C000051F8043B40F8043B51F8043B40F8043BA6
:104C100051F8043B40F8043B51F8043B40F8043B96
:104C200051F8043B40F8043B403ABDD2303211D336
:104C300051F8043B40F8043B51F8043B40F8043B76
:104C400051F8043B40F8043B51F8043B40F8043B66
:104C5000103AEDD20C3205D351F8043B40F8043B36
:104C6000043AF9D2043208D0D2071CBF11F8013B34
:104C700000F8013B01D30B8803806046704700BFFA
:104C8000082A13D38B078DD010F003038AD0C3F109
:104C90000403D21ADB071CBF11F8013B00F8013BEB
:104CA00080D331F8023B20F8023B7BE7043AD9D3AA
:104CB000013A11F8013B00F8013BF9D20B7803707F
:104CC0004B7843708B78837060467047F0B5304BFB
:104CD0001B681B06FBD42F4B1B6813F08002F6D118
:104CE00072B62D4B1978002950D02C4908684F68AE
:104CF0008E68CD680C693844143130440968284402
:104D000020440844C0F34E00254940F400400860A8
:104D1000C86A0F6B4E6B8D6BCC6B3844403130449E
:104D20000968284420440844C0F34E001D4940F45B
:104D30000040086001F10811143151F8140C51F8C9
:104D4000107C51F80C6C51F8085C51F8044C09685F
:104D500038443044284420440844C0F34E001249EB
:104D600040F400400860C86A0F6B4E6B8D6BCC6BD3
:104D70003844403130440968284420440844C0F392
:104D80004E000A4940F4004008601A7062B6F0BD57
:104D900024B0034024B00B40F988FF1F38B0034013
:104DA0002CB0034030B003402CB00B4030B00B406F
:104DB00010B5204B2048214960221A70E1225A7018
:104DC0001F4B204A1C78204B082C01D1012402E003
:104DD0000A2C03D139240460132005E00C2C0CBFED
:104DE00035243D2404601220086014601860174BBD
:104DF00017491B78174A03B101230B601360164B48
:104E0000164A1978164B012901D880210BE0042994
:104E100001D8842107E0082901D8852103E0102961
:104E200094BF86218721116019600E4B01221A70F0
:104E300010BD00BF0040074008B003400CB0034065
:104E40006487FF1F08B00B400CB00B40FC88FF1FAD
:104E500020B0034020B00B406587FF1F24B0034003
:104E600024B00B40F988FF1F0C2804D9102828BF54
:104E70001020102307E00A2804D8092834BF08238B
:104E80000A2300E00C23094AD9B2081A1070084A14
:104E90001078834208D0074B11701B7813B1064B72
:104EA00000221A60FFF784BF704700BFF888FF1F19
:104EB0006487FF1FF988FF1F24B0034010B5114B12
:104EC0001B7804460BB1FFF701FF012C0E4A01D8F5
:104ED000002302E0042C02D8042313600EE0082C07
:104EE00003D805231360082308E0102C03D80623F9
:104EF0001360102302E0072313602023034A13707A
:104F000010BD00BFF988FF1F24B003406587FF1F55
:104F10000D2838B50FD9172801D80E380AE0A0F1AE
:104F20001A03052B01D8093804E0A0F12203062B4F
:104F300047D81838C0B2244B1C5C244B1B780BB1EB
:104F4000FFF7C4FE210614D472B6214B214D1C601C
:104F500001232B7062B672B61D4B1B681A0601D571
:104F60001D4B1FE02B78002BEFD062B602F084FCC3
:104F7000F1E772B6194B1A4D1A6814F0400F14BFBE
:104F800022F0100242F010021A60164B04F03F02A9
:104F90001A6001232B7062B672B6124B1B681B0697
:104FA00008D5114B186800232B7062B60F4B1B7885
:104FB000184138BD2B78002BDCD062B602F05CFCC7
:104FC000EAE7002038BD00BF9AAD0000F988FF1F56
:104FD00000B00340FB88FF1F10B003400CB00B4033
:104FE000FA88FF1F00B00B4010B00B40F888FF1F7D
:104FF0000D2810B50FD9172801D80E380AE0A0F1F6
:105000001A03052B01D8093804E0A0F12203062B6E
:1050100027D81838C0B2134B1C5C134B1B780BB14C
:10502000FFF754FE230607D472B6104B44F0400439
:105030001C6001220E4B12E072B60E4B1A6814F07F
:10504000400F14BF22F0100242F010021A6004F068
:105050003F04094B44F040041C60084B01221A70C5
:1050600062B610BD9AAD0000F988FF1F00B0034082
:10507000FB88FF1F0CB00B4000B00B40FA88FF1FED
:105080000D280FD9172801D80E380AE0A0F11A030D
:10509000052B01D8093804E0A0F12203062B26D8FD
:1050A0001838C0B2134B1B56002B08DB124B1B6881
:1050B00013F0800F114B12D072B6114A07E0114B5A
:1050C0001B6813F0800F104B09D072B60F4A10689E
:1050D00000221A7062B60E4B1B78184170471B787D
:1050E000002B14BF4FF0FF306FF00100704700201D
:1050F000704700BF9AAD000000B00340FB88FF1F5F
:1051000010B0034000B00B40FA88FF1F10B00B40F6
:10511000F888FF1F084B1A6842F480521A60074B48
:105120001A78074B0AB1802200E0C0221A70054BA2
:1051300080F30C00188070472C800440FC88FF1F0F
:1051400021C00C4000C00C40024B1B78DB07FBD594
:10515000704700BF010002407FB5174B6A4603F15C
:1051600010056E4618685968144603C40833AB42EC
:105170002246F7D1114B1A7812F0020F1D4612D0B9
:1051800080229A7133229A7203225A7272B60C4CA0
:1051900046F001062046B04762B6237813F070034C
:1051A00001D0237006E044F621632A78D20701D4A7
:1051B000013BFAD104B070BDB2AD00000100024065
:1051C00000000240B0F5006F10B5044609D2064B4E
:1051D0001B78DB0701D4FFF7BFFF04F1A054207850
:1051E00010BD002010BD00BF0100024040F2FE7360
:1051F000984210B5044609D8054B1B78DB0701D44B
:10520000FFF7AAFF04F1A054208810BD002010BDB4
:1052100001000240024B187800F00100704700BF07
:1052200001000240B0F5006F38B504460D460FD2BC
:10523000084B1B78DB0701D4FFF78EFF04F1A05465
:105240002378AB4204D02570BDE83840FFF77CBF1F
:1052500038BD00BF0100024038B540F2FE739842ED
:1052600004460D461ED8104B1B78DB0701D4FFF710
:1052700073FF14F0010F04F1A05404D12388AB4252
:1052800010D025800AE02378AB4202D02570FFF7CA
:105290005BFF63782D0AAB4204D06570BDE83840EF
:1052A000FFF752BF38BD00BF01000240024B1A6831
:1052B00001321A60704700BF0089FF1F08B50B4C10
:1052C0002368580301D501F0A3FB2368590501D5D4
:1052D00000F0CAFC23681A0501D500F0A7FF236877
:1052E000DB04ECD501F010FAE9E700BF348004409C
:1052F00008B5FFF7E3FFFFFF014B10221A8070474C
:10530000002005407047FFFF024A136818441060F0
:10531000184670476887FF1F002070474FF0FF3026
:1053200070474FF0FF307047FEE7FFFFEFF3138346
:105330009BB9EFF3108098B9EFF3058323B10F2BDE
:1053400004D9084A985C01E04FF48070EFF31183B0
:105350003BB1834238BF184670474FF0FF3070476B
:1053600018467047F0E300E0044B054900221A603C
:105370000A60044A106010221A60704714D003407B
:1053800004D0034000D003402DE9F04105460E460D
:1053900008462E4902F092FD2D4B002847F61228B0
:1053A00014BF0227012708BF9846002428FA04F0FA
:1053B00002F08EFB4FF05E5102F0E2FB01463046F8
:1053C00002F090FD10B90134072CEFD128FA04F057
:1053D00002F07EFB314602F087FC4FF07C5102F078
:1053E000C5FA02F0B9FD4FF6FF73984228BF184680
:1053F000EB1E012B06D8174B174900221A600A60D2
:10540000164A1BE0A5F10903012B06D9A5F11403E7
:10541000032B02D96B1F012B06D8114B1149002217
:105420001A600A60104A09E0202D01D0192D0BD115
:105430000E4B0F4900221A600A600E4A04F007045E
:1054400044EAC70710601F60BDE8F081001BB74049
:10545000006CDC020090034004900340089003407D
:1054600000800340048003400880034000800B401C
:1054700004800B4008800B40212810B518D80D4A35
:1054800052F8303093F880423CB1012211B183F8D8
:10549000802010BD83F8002110BD02EBC0004368DE
:1054A0001A6811B142F0030201E022F002021A6010
:1054B00010BD00BFC4AD0000212816D80B4A02EB76
:1054C000C00301295B6852F8302004D182F88012B1
:1054D0004FF4A27208E0002082F8800211B94FF464
:1054E000807201E040F203121A607047C4AD000000
:1054F000282838B5604A04460B4611D112780B2A89
:1055000004D8C2F10C0201FA02F304E00C2A1CBF19
:105510000C3A41FA02F31846BDE83840FFF7FABDED
:1055200011780125002B05FA01F2D8BF002102DD18
:10553000934205D32946FFF79FFF2046294697E06F
:105540000338C2B2012A01D84C4A06E0202C01D00F
:10555000192C01D14A4A00E04A4A126802FB033280
:10556000CA401D287BD8DFE800F0575F4E337A7AB7
:10557000212A7A7A7A7A7A7A7A7A7A3C450F187A74
:10558000707A7A7A7A7A7A673F4B1A6003F59733A2
:1055900040F2444203F5FA735FE03C4B1A6003F5B6
:1055A000973340F2444203F5F87356E0384B1A60E3
:1055B00003F5973340F2444203F5F6734DE0354B63
:1055C0001A6003F5973340F2444203F5F47344E064
:1055D000314B1A6003F59F3340F2444203F5F073F8
:1055E0003BE02E4B1A6003F59F3340F2444203F533
:1055F000EE7332E02A4B1A6003F59F3340F24442C7
:1056000003F5EC7329E0274B1A6003F59F3340F252
:10561000444203F5EA7320E0234B1A6003F580331C
:105620004FF45172203318E0204B1A6003F5803399
:105630004FF451721C3310E01D4B1A60A3F5DB23AD
:105640004FF45172A3F5F96307E01A4B1A60A3F502
:10565000DB234FF45172A3F2CC731A6038BD7F2B59
:105660002046D4BF00210121FFF706FF204601217B
:10567000BDE83840FFF720BF6C87FF1F089003404C
:1056800008800B40088003401080034018800340CE
:10569000208003402880034030800340388003404E
:1056A000408003404880034010900340189003401E
:1056B00010800B4018800B4072B60B4B0B491A68D8
:1056C0000B4B1B68096862B6490102D5322A88BFB4
:1056D0000133C2F5BB326021FF32B2FBF1F24FF46D
:1056E0007A7000FB0320704718E000E004ED00E052
:1056F0000089FF1F38B50446FFF7DEFF054624B9D1
:1057000038BD013C0AD005F57A75FFF7D5FF401B7F
:10571000B0F57A7FF5D202F0AFF8F6E738BDFFFFBB
:105720001F4B4FF4000210B51A604FF080721A60E0
:105730004FF000721A604FF080621A604FF0006202
:105740001A60184B184A194C00204BF6FF7118606C
:10575000596028231360936013619361136293620D
:10576000136393630922226004F58054043420609B
:105770006160A360236144F8042C04F5FE242060DA
:105780000B4801600B490B608B600B4B1A60FFF7F5
:105790000FFBFA20FFF7AEFFBDE8104001F036BC6A
:1057A00008E100E0048003400C80034000800340D7
:1057B00008800B400C800B4000800B401D4B1A688A
:1057C00042F480621A601C4A002313801B4A138033
:1057D0001B4A13701B4A13701B4A13701B4B40F279
:1057E00013321A604FF451725A60194BC0F34432AD
:1057F0001A70C0F347125A700221042200F01F00F1
:1058000098729A70D9745A7588221A743C22DA7088
:105810009A7842F0A0029A709A7902F0DF029A71A7
:105820000C4B40226FF44A711A700B444FF4005233
:105830001A607047348004408C8AFF1F0A89FF1F5A
:10584000948AFF1F8E8AFF1F0889FF1F40A0044013
:1058500000A006402DE400E0134A937800F0030115
:1058600003F0EC030B43410748BF43F01003937070
:1058700000F00F03042B0C4903D18B7943F0400354
:105880008B715379C20603F0EF03074A48BF43F018
:10589000100353719379810603F0EF0348BF43F07F
:1058A00010039371704700BF00A0064008B5114B6C
:1058B0001B685B0500D408BD0F4B1A7802F0FF038C
:1058C00012B101F0D9FFF7E70C4A4FF40051116013
:1058D0000B4A0C49D37040F203120A604A600A4A2C
:1058E00013800A4A13800A4B1B680BB101221A70FD
:1058F00008BD00BF348004400889FF1F84E100E038
:1059000000A0064040A004408C8AFF1F0A89FF1FA8
:105910000489FF1F38B50446094B1B7803F0FF05C7
:10592000002BF9D120460121FFF7C6FD204629466C
:10593000FFF7A2FD034B53F83420034B1A6038BD28
:105940000889FF1FC4AD0000908AFF1F0D4A38B5BB
:10595000146814F480624FF0000410D021280A4D1E
:105960000AD80A4A012152F830302B60FFF7A4FD13
:105970002B681C70012038BD2C60204638BD1046B5
:1059800038BD00BF348004400489FF1FC4AD00004F
:105990000E4B1B6813F4806316D012280C4B03D1F6
:1059A00040F202310B4A04E0142809D10A4A40F2BD
:1059B000023111605A7B42F001025A730120704794
:1059C0005A7B02F0FE025A73002070473480044074
:1059D00000A006400CA0044014C00440F8B51F4BC2
:1059E0001B685A05064638D51D4B1B680BB10122B2
:1059F0001A701C4B9A7942F020029A711A4B1C784B
:105A00000134802C1F4628BF0024184D2B78A34258
:105A100018D1FFF78BFC40280FDC124A13791B06C4
:105A2000F3D52B7812490133802B28BF0023C95CA2
:105A3000DBB2C9B2D1712B70E7E7FF28E5DD01F0D9
:105A40001BFFE2E70A4BF6B21E550A4B01221A7001
:105A5000044BE4B2BC223C70DA70F8BD34800440E0
:105A6000908AFF1F00A00640948AFF1F8E8AFF1FA6
:105A70000C89FF1F0889FF1F294B1B685A052DE958
:105A8000F04707468A4649D5264B1B680BB10122D1
:105A90001A70254B9A7942F020029A713D4607EB25
:105AA0000A039D4237D2DFF89080204E98F80040DC
:105AB00096F800900134802C28BF00245FFA89F901
:105AC000A1451DD1184BBC22DA70FFF72FFC4028EE
:105AD0000FDC154A13791B060FD5337814490133AF
:105AE000802B28BF0023C95CDBB2C9B2D1713370EF
:105AF00003E0FF2801DD01F0BFFE33784B45E4D021
:105B00000B4B15F8012B1A550A4B0122E4B21A70FF
:105B100088F80040C3E7044BBC22DA70BDE8F08788
:105B200034800440908AFF1F00A006408E8AFF1F29
:105B30000C89FF1F0889FF1F948AFF1F08B5034BBC
:105B40001B7813B101F098FEF9E708BD0889FF1F23
:105B5000064A074B1B781078DBB2C0B283422CBFD9
:105B60007F3000F1FF30C01A704700BF8E8AFF1FE0
:105B7000948AFF1F054B1888054B1B8880B29BB287
:105B8000984238BF00F58070C01A70478C8AFF1F9A
:105B90000A89FF1F114B12491A880B8892B29BB2D7
:105BA0009A4210B516D00133B3F5807F28BF002389
:105BB0000C489CB2C05C0C800B490968C0B259B15A
:105BC0009A4238BF02F58072D31A1A2B04DC0023E4
:105BD0000B7010BD4FF0FF3010BD00BF8C8AFF1F4F
:105BE0000A89FF1F8C89FF1F0489FF1F094B1A8830
:105BF000094B1B8892B29BB29A4208D00133B3F58D
:105C0000807F28BF0023054AD05CC0B270474FF0A8
:105C1000FF3070478C8AFF1F0A89FF1F8C89FF1F86
:105C20000C4B1B685B0514D50B4BDA7802F0CB02EA
:105C3000DA7040225A74DA7842F03402DA70074B94
:105C40001A88074B92B21A80064B1B680BB10022D0
:105C50001A7070473480044000A006400A89FF1F74
:105C60008C8AFF1F0489FF1F30B53E4B1A7912F052
:105C7000300F32D072B69A7D02F0FF0022B9DA7985
:105C800040225A7462B628E062B6374A3749138810
:105C900009889BB289B21446324AD5795A1CB2F5AA
:105CA000807F28BF00228A42EDB202D0304B9D5443
:105CB0001346421E12F0FF00EED19AB222802D4A06
:105CC000126852B18B4236BFC1F58071C1EB03033C
:105CD0005B18272BC4BF01231370224BD978C9B29C
:105CE0000A0620D51B791D061DD5234B234A1D7896
:105CF0001378EDB2DBB21046AB420CD0194A013337
:105D0000802B14791E4C28BF0023E45CE4B2D471CC
:105D1000127D072AF0D9DBB20370124B1A791406F0
:105D200044BF7C22DA700F4B9A7C500706D5154A87
:105D300010780130C0B2107004229A74490610D550
:105D4000084B1A7952060CD50F4A002111700F4AE0
:105D5000126802B111709A7902F0DF029A713C2246
:105D6000DA7030BD00A006408C8AFF1F0A89FF1F31
:105D70008C89FF1F0489FF1F948AFF1F8E8AFF1FD3
:105D80000C89FF1F0091FF1F0889FF1F908AFF1FCA
:105D90001D4B1A6842F400621A601C4A00231380EB
:105DA0001B4A13801B4A13701B4A13701B4A137043
:105DB0001B4B40F213321A604FF451725A60194B68
:105DC000C0F344321A70C0F347125A7000F01F003B
:105DD0000422022198729A70D9745A7588221A7412
:105DE0003C22DA709A7842F0A0029A709A7902F016
:105DF000DF029A710C4B40221A70A3F22B334FF43E
:105E000000421A60704700BF34800440A08CFF1F1E
:105E10009E8AFF1FA88CFF1FA28CFF1F9C8AFF1F5A
:105E20000CB0044000B006402FE400E0134A937821
:105E300000F0030103F0EC030B43410748BF43F0BC
:105E40001003937000F00F03042B0C4903D18B79DE
:105E500043F040038B715379C20603F0EF03074A06
:105E600048BF43F0100353719379810603F0EF03A9
:105E700048BF43F010039371704700BF00B0064065
:105E800008B5114B1B681B0500D408BD0F4B1A78D1
:105E900002F0FF0312B101F0EFFCF7E70C4A4FF4F8
:105EA000004111600B4A0C49D37040F203120A60A2
:105EB0004A600A4A13800A4A13800A4B1B680BB1D6
:105EC00001221A7008BD00BF348004409C8AFF1F65
:105ED00084E100E000B006400CB00440A08CFF1F3D
:105EE0009E8AFF1F988AFF1F38B50446094B1B780E
:105EF00003F0FF05002BF9D120460121FFF7DCFA62
:105F000020462946FFF7B8FA034B53F83420034BD9
:105F10001A6038BD9C8AFF1FC4AD0000A48CFF1F0F
:105F20000D4A38B5146814F400624FF0000410D024
:105F300021280A4D0AD80A4A012152F830302B6034
:105F4000FFF7BAFA2B681C70012038BD2C60204680
:105F500038BD104638BD00BF34800440988AFF1F0A
:105F6000C4AD00000B4B1B6813F4006310D017285E
:105F7000094B09D1094A40F2023111605A7B42F0C3
:105F800001025A73012070475A7B02F0FE025A73D5
:105F9000002070473480044000B0064008B0044040
:105FA000F8B51F4B1B681A05064638D51D4B9A7964
:105FB00042F020029A711C4B1B680BB101221A702F
:105FC0001A4B1C780134802C1F4628BF0024184D22
:105FD0002B78A34218D1FFF7A9F940280FDC114A0A
:105FE00013791B06F3D52B7812490133802B28BF78
:105FF0000023C95CDBB2C9B2D1712B70E7E7FF287F
:10600000E5DD01F039FCE2E70A4BF6B21E550A4B1A
:1060100001221A70034BE4B2BC223C70DA70F8BD66
:106020003480044000B00640A48CFF1FA88CFF1FE2
:10603000A28CFF1FA08AFF1F9C8AFF1F294B1B6891
:106040001A052DE9F04707468A4649D5264B9A7925
:1060500042F020029A71254B1B680BB101221A7085
:106060003D4607EB0A039D4237D2DFF89080204E71
:1060700098F8004096F800900134802C28BF002446
:106080005FFA89F9A1451DD1174BBC22DA70FFF7E1
:106090004DF940280FDC144A13791B060FD53378CD
:1060A00014490133802B28BF0023C95CDBB2C9B27D
:1060B000D171337003E0FF2801DD01F0DDFB33789F
:1060C0004B45E4D00B4B15F8012B1A550A4B012216
:1060D000E4B21A7088F80040C3E7034BBC22DA70C0
:1060E000BDE8F0873480044000B00640A48CFF1F58
:1060F000A28CFF1FA08AFF1F9C8AFF1FA88CFF1F76
:1061000008B5034B1B7813B101F0B6FBF9E708BDE6
:106110009C8AFF1F064A074B1B781078DBB2C0B27F
:1061200083422CBF7F3000F1FF30C01A704700BFA0
:10613000A28CFF1FA88CFF1F054B1888054B1B88DE
:1061400080B29BB2984238BF00F5C070C01A704749
:10615000A08CFF1F9E8AFF1F114B12491A880B88C3
:1061600092B29BB29A4210B516D00133B3F5C07FFC
:1061700028BF00230C489CB2C05C0C800B49096806
:10618000C0B259B19A4238BF02F5C072D31A1A2B65
:1061900004DC00230B7010BD4FF0FF3010BD00BFBA
:1061A000A08CFF1F9E8AFF1F208BFF1F988AFF1F56
:1061B000094B1A88094B1B8892B29BB29A4208D0AD
:1061C0000133B3F5C07F28BF0023054AD05CC0B2BD
:1061D00070474FF0FF307047A08CFF1F9E8AFF1F53
:1061E000208BFF1F0C4B1B681B0514D50B4BDA785B
:1061F00002F0CB02DA7040225A74DA7842F03402AC
:10620000DA70074B1A88074B92B21A80064B1B684C
:106210000BB100221A7070473480044000B0064071
:106220009E8AFF1FA08CFF1F988AFF1F30B53E4B30
:106230001A7912F0300F32D072B69A7D02F0FF0058
:1062400022B9DA7940225A7462B628E062B6374A37
:106250003749138809889BB289B21446324AD579E6
:106260005A1CB2F5C07F28BF00228A42EDB202D08C
:10627000304B9D541346421E12F0FF00EED19AB2ED
:1062800022802D4A126852B18B4236BFC1F5C071CF
:10629000C1EB03035B18272BC4BF01231370224BF0
:1062A000D978C9B20A0620D51B791D061DD5234B06
:1062B000234A1D781378EDB2DBB21046AB420CD006
:1062C000194A0133802B14791E4C28BF0023E45C4B
:1062D000E4B2D471127D072AF0D9DBB20370124BFD
:1062E0001A79140644BF7C22DA700F4B9A7C50074F
:1062F00006D5154A10780130C0B2107004229A7485
:10630000490610D5084B1A7952060CD50F4A0021C0
:1063100011700F4A126802B111709A7902F0DF020F
:106320009A713C22DA7030BD00B00640A08CFF1F8D
:106330009E8AFF1F208BFF1F988AFF1FA88CFF1FBC
:10634000A28CFF1FA08AFF1FC388FF1F9C8AFF1F0C
:10635000A48CFF1F174B1A6842F480521A60164A29
:1063600000231380154A1380154A1380154A1380A1
:10637000154A1370154A40F2133111604FF45171F0
:106380005160134AC0F344311170C0F3471100F05B
:106390001F0051709072937013742C23D3700D4BA7
:1063A00040226FF44B711A700B444FF400321A60A4
:1063B000704700BF34800440B48FFF1FB28CFF1FB2
:1063C000BC8FFF1FB68FFF1FB08CFF1F08C004409B
:1063D00000C0064031E400E0134A937800F0030166
:1063E00003F0EC030B43410748BF43F010039370E5
:1063F00000F00F03042B0C4903D18B7943F04003C9
:106400008B715379C20603F0EF03074A48BF43F08C
:10641000100353719379810603F0EF0348BF43F0F3
:1064200010039371704700BF00C0064008B5114BC0
:106430001B68DB0400D408BD0F4B1A7802F0FF0381
:1064400012B101F019FAF7E70C4A4FF4003111606C
:106450000B4A0C49D37040F203120A604A600A4AA0
:1064600013800A4A13800A4B1B680BB101221A7071
:1064700008BD00BF34800440B08CFF1F84E100E001
:1064800000C0064008C00440B48FFF1FB28CFF1F3D
:10649000AC8CFF1F38B50446094B1B7803F0FF0591
:1064A000002BF9D120460121FFF706F820462946A6
:1064B000FEF7E2FF034B53F83420034B1A6038BD5C
:1064C000B08CFF1FC4AD0000B88FFF1F0D4A38B558
:1064D000146814F480524FF0000410D021280A4DA3
:1064E0000AD80A4A012152F830302B60FEF7E4FF47
:1064F0002B681C70012038BD2C60204638BD10462A
:1065000038BD00BF34800440AC8CFF1FC4AD000018
:106510000B4B1B6813F4805310D00E28094B09D184
:10652000094A40F2023111605A7B42F001025A736B
:10653000012070475A7B02F0FE025A730020704718
:106540003480044000C0064004C00440F8B51F4B2E
:106550001B68DA04064638D51D4B1B680BB10122B7
:106560001A701C4B1C88A4B20134B4F5C07F1F46BE
:1065700028BF0024184D2B889BB2A3421AD1FEF7E6
:10658000D5FE402811DC154A13791B06F2D52B885D
:1065900013499BB20133B3F5C07F28BF0023C95C08
:1065A0009BB2C9B2D1712B80E4E7FF28E2DD01F094
:1065B00063F9DFE70A4BF6B21E550A4B01221A7047
:1065C000064BA4B2AC223C80DA70F8BD34800440A3
:1065D000B88FFF1FBC8FFF1FB68FFF1F00C0064084
:1065E000B48CFF1FB08CFF1F38B504464518AC4271
:1065F00004D014F8010BFFF7A9FFF8E738BDFFFF3F
:1066000008B5034B1B7813B101F036F9F9E708BD63
:10661000B08CFF1F064A074B1B8810889BB280B2C4
:1066200083422CBF00F27F1000F1FF30C01A704788
:10663000B68FFF1FBC8FFF1F054B1888054B1B88AB
:1066400080B29BB2984238BF00F5C070C01A704744
:10665000B48FFF1FB28CFF1F114B12491A880B8891
:1066600092B29BB29A4210B516D00133B3F5C07FF7
:1066700028BF00230C489CB2C05C0C800B49096801
:10668000C0B259B19A4238BF02F5C072D31A1A2B60
:1066900004DC00230B7010BD4FF0FF3010BD00BFB5
:1066A000B48FFF1FB28CFF1F348EFF1FAC8CFF1FF7
:1066B000094B1A88094B1B8892B29BB29A4208D0A8
:1066C0000133B3F5C07F28BF0023054AD05CC0B2B8
:1066D00070474FF0FF307047B48FFF1FB28CFF1F21
:1066E000348EFF1F054B1A88054B92B21A80054B5A
:1066F0001B680BB100221A70704700BFB28CFF1FDD
:10670000B48FFF1FAC8CFF1F10B5314B1A79920666
:1067100023D5304AD87913882F499BB20133098891
:10672000B3F5C07F28BF002389B28B42C0B203D02B
:106730002A49C85499B21180294A116869B1294A75
:10674000128892B2934236BFC2F5C072C2EB030305
:106750009B18272BC4BF01230B701D4AD178C9B2E7
:106760000C0618D51379180615D51F4B1D481C8823
:106770000388A4B29BB29C4202D16C23D3700AE07E
:106780000133B3F5C07F28BF0023184CE45C9BB2F3
:10679000E4B2D47103800E4B9A7C520706D5144A9A
:1067A00010780130C0B2107004229A744B060ED5D6
:1067B000074B1A7912F0400F194608D00D4B0022F2
:1067C0001A700D4B1B6803B11A702C23CB7010BDCF
:1067D00000C00640B48FFF1FB28CFF1F348EFF1F16
:1067E000AC8CFF1FB68FFF1FBC8FFF1FB48CFF1F29
:1067F0000191FF1FB08CFF1FB88FFF1F21282BD8DE
:10680000164B1B5CFF2B27D0154A02EBC000002162
:1068100042681160134A106840F020001060124A6C
:1068200001201160114998400860114841F8040C9A
:10683000104911604FF4A07101397FF4FDAF116868
:106840008905FCD42022013A7FF4FDAF0A4A1BB22D
:1068500032F8130080B2704700207047D4AE0000B9
:10686000C4AD00003880044000500440085004408B
:106870000000020380014A0000510440F0B50C4BB7
:106880000C4C1A7842F0020504EBC50682F00102B6
:10689000706009481A700678002E0CBF8827C82738
:1068A00086F0010647EA0141067044F83510F0BD54
:1068B0002890FF1F0080FF1FA090FF1F431E032B87
:1068C00010B510D872B6094A52F8230048B1416891
:1068D00042F82310064A018832F81340611A22F860
:1068E000131062B610BD002010BD00BF1890FF1F2E
:1068F0000291FF1F013803280AD872B6054B53F8DE
:106900002030002013B101305B68FBE762B67047AE
:10691000002070476C90FF1F10B572B60123174A14
:106920001A4412F8012C12071CD59900144A52F887
:1069300031402CB902EB431308305860114B09E089
:1069400041F0010152F8314064B902EBC103083053
:1069500058600D4B42F831300C4B1A78013A1A70DE
:1069600062B610BD0133052BD9D162B6074B0022A8
:106970001A70BDE8104000F0A7BB00BF28B00000AF
:106980000080FF1F88004000C80040009690FF1F55
:10699000431E032B30B532D8194A400140F0100095
:1069A000104472B6174CE25C032A09D8DFE802F003
:1069B000160218050830022213E00830042210E005
:1069C0001148124A50F8234014B940F8231002E04D
:1069D00052F82300416042F823100FE0032200E048
:1069E0000522E25410F0080F01F108030A88436001
:1069F0000CBF8823C82343EA0243036062B630BD5C
:106A00000080FF1FD48FFF1F6C90FF1F7C90FF1F23
:106A10002DE9F84FAB4F3C78E4B214F0040F3D463B
:106A200019D0A94B1B78A3B1A84A117801F0FF0334
:106A300021B1013BDBB2137003B900BEA44A117847
:106A400001F0FF0329B1013BDBB213700BB900F079
:106A50004FFC04233B7004F0080303F0FF02002BFB
:106A600000F067829B4B9C4C1A78D2B215094FEA12
:106A7000920840F0E48104EBC803596854F83830B8
:106A8000C3F38303013B0C2B00F2D681DFE813F044
:106A900095019501D401D401D401D401D401D401CC
:106AA000B001D401D401D4010D008C4D0A684B68AB
:106AB0008B486B6001218B4B44F838302A60DFF83B
:106AC0005082017092B240F2816000238242C8F885
:106AD00000302361A36117D8B2F5D06F80F01E811A
:106AE000B2F5817F00F0CF8006D8802A00F0BA800E
:106AF000822A00F0BB8031E140F202339A4200F07A
:106B0000D180B2F5A06F1CE042F22100824200F079
:106B100051810ED8B2F5086F00F09E80B2F5106F6B
:106B200040F01C81684B6C4EAA781A7006F18009FF
:106B30000AE042F221218A4200F0088142F2213328
:106B40009A4200F00F8109E1336A1B0603D5706A8F
:106B5000083800F0B9FA08364E45F5D10026B1469E
:106B6000DFF8B0A156F80A0028B1D0F804B000F060
:106B7000ABFA5846F8E74AF806005B4BDFF898A1F5
:106B8000F05056F80A0028B1D0F804B000F09CFA92
:106B90005846F8E7554B4AF80600F050544B23F896
:106BA0001900544B19F80320023A032A08D8DFE8E9
:106BB00002F002040204002200E0012203F809208E
:106BC00009F10109B9F1040F06F10406C8D14A4BD5
:106BD00000221A7001269A46484A494B32443344EF
:106BE00012F8012C9B0012F0080F1A704FEA860968
:106BF00025D000F04BFA38B104EB4613083058604A
:106C0000404B44F8393006E09AF8003044F8390037
:106C100001338AF8003000F039FA49F0010338B145
:106C200004EBC302083050602E4A44F8332006E0DB
:106C300044F833009AF8003001338AF8003049F004
:106C40000202013649F003090023052E44F83230D0
:106C500044F83930C0D186E01B4B2B4C1B78237095
:106C60000B4683E0284C237063707EE0AA88042AD8
:106C700074D8254C920023706370244B9B5C9E0754
:106C800073D5217071E0AA8802F07F02042A65DCC6
:106C90006B88002B62D191001C4A0A44117821F0C4
:106CA000020159E0AA8802F07F02042A56DC6B88B0
:106CB000002B53D19100154A0A44117841F002018A
:106CC0004AE000BF802007409F90FF1F2990FF1FD0
:106CD000A190FF1F902007400080FF1F8C90FF1F96
:106CE000A090FF1FC8004000C48FFF1F7C90FF1FB3
:106CF0000291FF1FD48FFF1F9690FF1F28B0000046
:106D000030C80110880040009790FF1FC020074046
:106D1000C08FFF1F1890FF1F6C90FF1F6A88A98803
:106D20009F4B53F8084CA3F10C00BCB133F80C6C2A
:106D3000964209D133F80A6C8E4205D1120A032A11
:106D40000CBF2378038911E00C33EAE7954A1168F8
:106D5000954A1160A978954A117004E0944B0F226E
:106D60001A7027E000231C4600E00223EE88B3429D
:106D700038BF1E46402E34BF3546402520462946A2
:106D8000FFF77CFD761B2C4403D1402D12D13546F4
:106D900003E0402E34BF3546402520462946FFF704
:106DA0006DFD761B2C4401D1402D03D1814AC8F8DA
:106DB000004016800122804B3DE0804B1A8842F251
:106DC00021039A4210D100237D4AC85C98540133B4
:106DD000072BF9D11368862B02D17A4B0F221A7038
:106DE00000200146FFF74AFD774B44F8383023E096
:106DF000764E3568B5B1DFF8BC81B8F80090B9F1CE
:106E0000400F34BF4C46402428462146FFF736FD4C
:106E1000C4EB09039BB2A8F800300BB9402C00D199
:106E20002B193360654B1A88B2F5A06F04D100228C
:106E30005A709A78664B1A7001225F4B6CE004EB33
:106E4000C806013D736802F00802A3F10800EDB224
:106E500002F0FF01002A36D000F036F95D485E4BA3
:106E600050F82520EAB1516840F8251002F10801D8
:106E70007160595D03290BD8DFE801F002040608B0
:106E8000032104E0022102E0052100E0042159551C
:106E900016F0080F12880CBF8823C82343EA024368
:106EA00042E05A5D032A07D8DFE802F040400204BE
:106EB000002206E0012204E016F0080F0CBF0222B7
:106EC00003225A5532E054F83820120C23F8082CCB
:106ED00022B3DFF834E123F8061C43F8041C5EF803
:106EE00025303E4913B94EF8250002E051F825300F
:106EF00058603B4B41F8250033F815100A4423F83D
:106F0000152000F0C3F810B10830706006E0354B72
:106F100044F838001A7801321A7007E02A4B324AD6
:106F200016F0080F08BF134644F8383008233B70AA
:106F300070E5E0071FD520492B482C4C02230B702D
:106F40002B4B1A702B4B186098602B48D8601A6135
:106F50009A615C60164B0D2018702848FF2303705F
:106F60002B700274264A1370264B9F221A7001233D
:106F70000B70BDE8F88F210604D50D4B0D221A7059
:106F800080232B70A20705D51C4B1A78D2B21A7039
:106F900002232B70E30644BF10232B70BDE8F88F4B
:106FA00038B000000089FF1F1491FF1FB090FF1F31
:106FB000C02007409490FF1F942007408C90FF1F33
:106FC0000C91FF1F2990FF1FC8004000C08FFF1FBA
:106FD000982007406C90FF1FD48FFF1FC48FFF1FA6
:106FE0000291FF1F9690FF1F88004000D88FFF1F5F
:106FF0002890FF1F0080FF1F2C90FF1F8820074054
:107000008C200740842007401890FF1F08B500F02F
:1070100071FC00221A4B0021D15098180832882A9E
:107020004160F7D1174A106840F48020106002F5E3
:1070300028326832C3F307201070C3F307401B0ED9
:1070400010751376FF2302F81C3C02F8143C02F87A
:107050008C3C012302F8083C82F8641002F8183CCA
:10706000094B70226FF450711A700B444FF4007288
:107070001A6003F1C04303F5C82310221A7008BD3B
:107080000080FF1F3480044049E400E072B60C4ADF
:107090001168B1FA81F30B2B02D962B60020704758
:1070A0004FF00040D84021EA0001116062B6054966
:1070B00048225343C8180022CA504260704700BF9C
:1070C0007087FF1F0084FF1F0C4B4822C31AB3FBBD
:1070D000F2F30B2B11D80A4A127822B1094A12781E
:1070E0000AB1FFF719BC72B6074A4FF0004121FA06
:1070F00003F311681943116062B670470084FF1FE3
:107100009690FF1F9F90FF1F7087FF1F10B5104CB8
:1071100023686BB120684288531C0244147A0288A9
:10712000934212D3FFF7D0FF094B00221A600DE003
:10713000084B1B7813B94FF0FF3010BD0320FFF749
:10714000BDFB20600028E5D1F5E74380204610BD57
:10715000AC90FF1F9F90FF1F10B50B4C236813B11D
:1071600023686BB902E0094B1B7813B94FF0FF306D
:1071700010BD0320FFF7A2FB20600028F0D1F5E747
:107180005A881344187A10BDAC90FF1F9F90FF1FC0
:10719000044B9888044B1B681BB11A885B88D31A70
:1071A000184470470291FF1FAC90FF1F2DE9F84370
:1071B0002D4E012307460C463370002C4FD02B4D2B
:1071C0002B68A9462BBB4AF2F928294B1B7803F000
:1071D000FF020BB9327015E00420FFF78BFB072884
:1071E00008D801233370FFF751FFC9F8000080B9B8
:1071F0001D4B1870B8F101081E4B01D01A782AB146
:1072000001221A704FF0FF30BDE8F88300F034FB24
:10721000DBE72968174A488800231370C0F1400251
:10722000944238BF224600F1080C10448C44488038
:10723000A41A934204D0F85C0CF803000133F8E779
:107240001F444B883F2B06D940230B800420FFF7B7
:107250009FFB00232B60084B05221A70ADE73470AA
:107260002046BDE8F88300BFA290FF1FA490FF1F37
:107270009F90FF1FA890FF1FA190FF1F07B502ABB3
:10728000012103F8010D1846FFF790FF03B05DF8E8
:1072900004FBFFFF2DE9F041114B1B78F3B1114EB8
:1072A000114B3468114D01271F7098464CB10027CF
:1072B00063882F70042023802146FFF769FB376025
:1072C00009E0FFF7E3FE014620B104202C70FFF730
:1072D0005FFB00E02F70002388F80030BDE8F081EC
:1072E0009F90FF1FA490FF1FA290FF1FA190FF1F60
:1072F00038B50E4B1B7803F0FF05ABB90C4C216879
:1073000031B14B880B800420FFF742FB256038BD6C
:10731000FFF7BCFE014620B10420BDE83840FFF76E
:1073200037BB044B01221A7038BD00BFA290FF1F6B
:10733000A490FF1FA190FF1F08B50368C9B21B6886
:10734000984708BD08B50368C9B21B68984708BDCF
:1073500008B50368C9B21B68984708BD08B503683B
:10736000C9B21B68984708BD4B0803F1376000F5A8
:10737000D830B0FBF1F0FEF721BA10B54B0803F19D
:10738000376000F5D8301446B0FBF1F0FEF716FA7E
:107390002046BDE81040FEF75FBAFEF787BA084600
:1073A000FEF7B8BA08B50846FEF7D0FA003018BFA5
:1073B000012008BD08B50846FEF7EAFA003018BFFC
:1073C000012008BDFEF7D6BBFEF710BCFEF7E2BBFE
:1073D000FEF7B4BBFEF724BCFEF7BABB08B50846FF
:1073E000FEF7FCFA012008BD08B50846FEF7F6FADC
:1073F000012008BD10B5084614461146FEF73CFBB7
:10740000204610BD38B508460D4600F01EFF044664
:1074100021462846FEF730FB204638BD7047FFFF67
:10742000044B00221A714FF47A711A73024A996060
:107430001A607047B490FF1F00AF000008B50368E2
:10744000C9B21B68984708BD08B50368C9B21B6874
:10745000984708BD08B50368C9B21B68984708BDBE
:1074600008B50368C9B21B68984708BD4B0803F10B
:10747000376000F5D830B0FBF1F0FEF789BC10B5ED
:107480004B0803F1376000F5D8301446B0FBF1F03B
:10749000FEF77EFC2046BDE81040FEF7C7BCFEF7B5
:1074A000EFBC0846FEF720BD08B50846FEF738FDDC
:1074B000003018BF012008BD08B50846FEF752FD90
:1074C000003018BF012008BDFEF736BEFEF770BEC3
:1074D000FEF742BEFEF714BEFEF784BEFEF71ABEEC
:1074E00008B50846FEF75CFD012008BD08B5084652
:1074F000FEF756FD012008BD10B50846144611469A
:10750000FEF79CFD204610BD38B508460D4600F03C
:107510009CFE044621462846FEF790FD204638BDD5
:107520007047FFFF044B00221A714FF47A711A73EF
:10753000024A99601A607047C490FF1F58AF00005C
:1075400008B50368C9B21B68984708BD08B5036849
:10755000C9B21B68984708BD08B50368C9B21B6863
:10756000984708BD08B50368C9B21B68984708BDAD
:107570004B0803F1B76000F55840B0FBF1F0FEF79F
:10758000E9BE10B54B0803F1B76000F5584014464A
:10759000B0FBF1F0FEF7DEFE2046BDE81040FEF73E
:1075A0001BBFFEF743BF0846FEF774BF08B5084689
:1075B000FEF78CFF003018BF012008BD08B5084653
:1075C000FEF7A6FF003018BF012008BDFFF734B852
:1075D000FFF76EB8FFF740B8FFF712B8FFF782B8B1
:1075E000FFF718B808B50846FEF7B0FF012008BD40
:1075F00008B50846FEF7AAFF012008BD10B50846E9
:1076000014461146FEF7F0FF204610BD38B5084677
:107610000D4600F01AFE044621462846FEF7E4FF18
:10762000204638BD7047FFFF044B00221A714FF40B
:107630007A711A73024A99601A607047D490FF1FDA
:10764000B0AF000008B5F8F70DFFF9F7DDF800F06E
:1076500013F9FAE700F0D8BC00F0DEBC2DE9F041E8
:1076600000258C688AB0074688462E4694B12B4682
:10767000404601A9212200F0E6F83B68202C34BFE7
:10768000224620225B68384601A91544A41A98476F
:107690000644EBE730460AB0BDE8F08107B5064B7B
:1076A0001B88ADF80430036801A95B680222984783
:1076B00003B05DF804FB00BF00B0000008B503682C
:1076C0005B689847002008BD0EB403B503AA52F8C2
:1076D000041B019200F0AAFE02B05DF804EB03B0B7
:1076E000704770B505468AB022B90368C9B21B68F5
:1076F00098472CE0012A08BF0A2221B930228DF8D0
:107700002520212413E02124B1FBF2F002FB10110B
:10771000C9B209290AAE94BF303137312644C9B203
:1077200006F8241C014610B1013CE4B2ECE733B189
:10773000013CE4B20AAB23442D2203F8242C2B682D
:1077400001A95B6828462144C4F1220298470AB087
:1077500070BD0029BABF49422D2300230A22FFF73A
:10776000C0BFFFF715BDFFF7D1BCFFF7F5BCFFF7B2
:1077700091BD0846FFF782BD08461146FFF716BDCA
:107780007047FFFF044B00221A714FF47A711A738D
:10779000024A99601A607047E490FF1F10B0000021
:1077A00010B50446006800F037FC204610BD38B51F
:1077B00004460D460068013100F00EFD10B184E86A
:1077C0002100012038BD43688B4210B5044606D223
:1077D000FFF7EDFF20B1A3680BB9226813700120F9
:1077E00010BDF8B504460F46154622B9036803B12B
:1077F0001A7000230BE01146FFF7E5FF064640B97B
:10780000206810B100F008FC266000236360A360CC
:1078100004E0A5602068394600F00FFD2046F8BD61
:1078200038B50023044603604360836003730D464C
:1078300039B1084600F009FD294602462046FFF707
:10784000D0FF204638BD38B50C469AB191B1816859
:107850008B4202D30023237038BDC91A551E8D42B6
:1078600028BF0D4601682A461944204600F00CFD49
:107870000023635538BDFFFF10B50E4C2378BBB90C
:1078800001232370FFF784FC08B1FFF779FFFEF7AF
:1078900071F908B1FFF7C2FDFEF74EFC08B1FFF722
:1078A0003FFEFEF7C9FE08B1FFF7BCFE00232370C0
:1078B00010BD00BFF490FF1F10B50023B0FBF2F421
:1078C00002FB1400092894BF30303730C0B2C854CE
:1078D00020460CB10133F1E7CA18547022469A428F
:1078E00006DA885CCC5C8C54C8540132013BF6E764
:1078F000084610BD1FB572B6154B70221A70154A96
:10790000412111700F2102F8011C80221A701A788F
:107910001206FCD5104B186862B6104B984298BFFF
:107920000A2301AC98BF584321460A22FFF7C4FF3F
:107930000023E15C0A4A29B102EB430001330A2B20
:107940004180F6D101335B00137004B010BD00BF5D
:107950000000024007000240080002407F969800A5
:10796000FC87FF1F80F0004002E000BF81F0004173
:1079700042001FBF5FEA410392EA030F7FEA226CD5
:107980007FEA236C6AD04FEA1262D2EB1363C1BF65
:10799000D218414048404140B8BF5B42192B88BFD4
:1079A000704710F0004F40F4000020F07F4018BFF7
:1079B000404211F0004F41F4000121F07F4118BF17
:1079C000494292EA030F3FD0A2F1010241FA03FCBF
:1079D00010EB0C00C3F1200301FA03F100F00043A7
:1079E00002D5494260EB4000B0F5000F13D3B0F16F
:1079F000807F06D340084FEA310102F10102FE2ADE
:107A000051D2B1F1004F40EBC25008BF20F001004D
:107A100040EA03007047490040EB000010F4000FFB
:107A2000A2F10102EDD1B0FA80FCACF1080CB2EB8E
:107A30000C0200FA0CF0AABF00EBC25052421843ED
:107A4000BCBFD0401843704792F0000F81F4000192
:107A500006BF80F400000132013BB5E74FEA410365
:107A60007FEA226C18BF7FEA236C21D092EA030FD1
:107A700004D092F0000F08BF0846704790EA010F4B
:107A80001CBF0020704712F07F4F04D1400028BF78
:107A900040F00040704712F100723CBF00F500005A
:107AA000704700F0004343F0FE4040F40000704790
:107AB0007FEA226216BF08467FEA2363014642023C
:107AC00006BF5FEA412390EA010F40F4800070474F
:107AD0004FF0000304E000BF10F0004348BF4042F5
:107AE0005FEA000C08BF704743F0964301464FF031
:107AF00000001CE050EA010208BF70474FF000038D
:107B00000AE000BF50EA010208BF704711F00043CD
:107B100002D5404261EB41015FEA010C02BF84469D
:107B20000146002043F0B64308BFA3F18053A3F5FC
:107B30000003BCFA8CF2083AA3EBC25310DB01FA43
:107B400002FC634400FA02FCC2F12002BCF1004FC7
:107B500020FA02F243EB020008BF20F00100704758
:107B600002F1200201FA02FCC2F1200250EA4C00AC
:107B700021FA02F243EB020008BF20EADC707047F2
:107B80004FF0FF0C1CEAD0521EBF1CEAD15392EA00
:107B90000C0F93EA0C0F6FD01A4480EA010C4002DC
:107BA00018BF5FEA41211ED04FF0006343EA501036
:107BB00043EA5111A0FB01310CF00040B1F5000F78
:107BC0003EBF490041EAD3715B0040EA010062F127
:107BD0007F02FD2A1DD8B3F1004F40EBC25008BF11
:107BE00020F00100704790F0000F0CF0004C08BF2F
:107BF00049024CEA502040EA51207F3AC2BFD2F1FC
:107C0000FF0340EAC250704740F400004FF0000309
:107C1000013A5DDC12F1190FDCBF00F00040704743
:107C2000C2F10002410021FA02F1C2F1200200FA81
:107C300002FC5FEA310040F1000053EA4C0308BF48
:107C400020EADC70704792F0000F00F0004C02BF99
:107C5000400010F4000F013AF9D040EA0C0093F014
:107C6000000F01F0004C02BF490011F4000F013B6E
:107C7000F9D041EA0C018FE70CEAD15392EA0C0FDC
:107C800018BF93EA0C0F0AD030F0004C18BF31F047
:107C9000004CD8D180EA010000F00040704790F01D
:107CA000000F17BF90F0004F084691F0000F91F0C1
:107CB000004F14D092EA0C0F01D142020FD193EA87
:107CC0000C0F03D14B0218BF084608D180EA01000F
:107CD00000F0004040F0FE4040F40000704740F0EB
:107CE000FE4040F4400070474FF0FF0C1CEAD052B9
:107CF0001EBF1CEAD15392EA0C0F93EA0C0F69D015
:107D0000A2EB030280EA010C49024FEA402037D07F
:107D10004FF0805343EA111143EA10130CF0004076
:107D20008B4238BF5B0042F17D024FF4000C8B4266
:107D300024BF5B1A40EA0C00B3EB510F24BFA3EB46
:107D4000510340EA5C00B3EB910F24BFA3EB910316
:107D500040EA9C00B3EBD10F24BFA3EBD10340EA70
:107D6000DC001B0118BF5FEA1C1CE0D1FD2A3FF6B6
:107D700050AF8B4240EBC25008BF20F0010070476B
:107D80000CF0004C4CEA50207F32C2BFD2F1FF030E
:107D900040EAC250704740F400004FF00003013A3F
:107DA00037E792F0000F00F0004C02BF400010F4E3
:107DB000000F013AF9D040EA0C0093F0000F01F0F7
:107DC000004C02BF490011F4000F013BF9D041EA19
:107DD0000C0195E70CEAD15392EA0C0F08D142024C
:107DE0007FF47DAF93EA0C0F7FF470AF084676E71F
:107DF00093EA0C0F04D14B023FF44CAF08466EE7F8
:107E000030F0004C18BF31F0004CCAD130F00042C5
:107E10007FF45CAF31F000437FF43CAF5FE700BF1D
:107E20004FF0FF3C06E000BF4FF0010C02E000BF46
:107E30004FF0010C4DF804CD4FEA40024FEA4103E8
:107E40007FEA226C18BF7FEA236C11D001B052EA9E
:107E5000530C18BF90EA010F58BFB2EB030088BF64
:107E6000C81738BF6FEAE17018BF40F001007047D3
:107E70007FEA226C02D15FEA402C05D17FEA236CB5
:107E8000E4D15FEA412CE1D05DF8040B704700BFFC
:107E9000844608466146FFE70FB5FFF7C9FF002893
:107EA00048BF10F1000F0FBD4DF808EDFFF7F4FFCC
:107EB0000CBF012000205DF808FB00BF4DF808ED65
:107EC000FFF7EAFF34BF012000205DF808FB00BF88
:107ED0004DF808EDFFF7E0FF94BF012000205DF8AA
:107EE00008FB00BF4DF808EDFFF7D2FF94BF01205B
:107EF00000205DF808FB00BF4DF808EDFFF7C8FF54
:107F000034BF012000205DF808FB00BF4FEA4002AB
:107F1000B2F1FE4F0FD34FF09E03B3EB12620DD9B7
:107F20004FEA002343F0004310F0004F23FA02F021
:107F300018BF404270474FF00000704712F1610FC8
:107F400001D1420205D110F0004008BF6FF000409F
:107F500070474FF00000704742000ED2B2F1FE4F62
:107F60000BD34FF09E03B3EB126209D44FEA002308
:107F700043F0004323FA02F070474FF000007047CF
:107F800012F1610F01D1420202D14FF0FF30704770
:107F90004FF00000704700BF00210A2200F008BA2D
:107FA00000210A2200F004BA0A4603490346086881
:107FB000194600F06BB800BF7488FF1F70B50E4BF8
:107FC0000E4DED1AAD1000241E46AC4204D056F8FA
:107FD000242090470134F8E703F022F9084D094BBB
:107FE000ED1AAD1000241E46AC4204D056F82420F1
:107FF00090470134F8E770BD2CB200002CB20000AD
:1080000040B200002CB20000024B0146186800F09C
:108010008FB800BF7488FF1F024B0146186800F03C
:1080200043B800BF7488FF1F10B5C9B20244904224
:10803000034606D01C788C4200F10100F7D11846A7
:1080400010BD002010BD814270B501D300230EE0A9
:108050008C18A042FAD28518134613F1FF3305D3CA
:10806000514266182944F65CCE54F6E770BD93423F
:1080700003D0CC5CC4540133F9E770BD024403461D
:10808000934202D003F8011BFAE7704738B502FBB0
:1080900001F4214600F04CF8054618B100212246B3
:1080A000FFF7ECFF284638BD30B500293CD051F829
:1080B000042C0B1F1D49002AB8BF9B180A680C46E8
:1080C00012B95A600B6030BD93420DD2196858182E
:1080D000904203D15A581144426819605A60236093
:1080E00030BD994203D80A4651680029F9D1146875
:1080F00015199D420AD11B682344D0188842136089
:1081000012D10868034413604B680CE002D90C23B9
:10811000036030BD18681C188C4203D10C68496894
:10812000204418605960536030BD00BFFC90FF1FB1
:1081300070B5CD1C25F0030508350C2D38BF0C2576
:10814000002D06463FDB8D423DD3214B1C6818466F
:108150002146A1B10B685B1B0ED40B2B03D90B601E
:10816000CC18CD501FE08C4202D1626802601AE048
:108170004B6863600C4616E00C464968E9E7154C0D
:1081800023681BB9304600F031F82060294630469C
:1081900000F02CF8431C014615D0C41C24F0030445
:1081A00084420AD1256004F10B00231D20F0070052
:1081B000C31A0BD05A42E25070BD3046611A00F02B
:1081C00015F80130EED10C233360002070BD00BFE4
:1081D000FC90FF1FF890FF1F0A46034903460868FA
:1081E000194600F001BA00BF7488FF1F38B5064C6D
:1081F0000023054608462360FDF786F8431C02D19C
:10820000236803B12B6038BD1891FF1FC9B2024625
:1082100010F8013B1BB18B42F9D110467047002981
:10822000FBD01846704710F8012B11F8013B012ACA
:1082300028BF9A42F7D0D01A7047034611F8012B95
:1082400003F8012B002AF9D17047034613F8012BDC
:10825000002AFBD1181A0138704770B592B10B464D
:1082600005461C7810F8016BB44201F1010101D1FF
:10827000012A03D128781B78C01A70BD013A002C5E
:10828000EDD1F7E7104670BD10B5034632B111F8D5
:10829000014B03F8014B013A002CF7D11A449342E9
:1082A00003D0002103F8011BF9E710BD84463F48C5
:1082B0002DE9F04FD0F800800E46344614F8015BEB
:1082C00008EB0500407800F0080000F0FF0708B157
:1082D0002646F2E72D2D03D1B41C7578012703E063
:1082E0002B2D04BF7578B41C33F010000DD1302D48
:1082F00008D1207800F0DF00582851D1657810238C
:10830000023402E0002B08BF0A23002F0CBF6FF0DD
:10831000004A4FF0004ABAFBF3F9002603FB19AA02
:10832000304608EB050B9BF801B01BF0040F01D0A1
:10833000303D0BE01BF0030B1BD0BBF1010F14BF52
:108340004FF0570B4FF0370BCBEB05059D4210DA82
:10835000B6F1FF3F0AD0484506D801D1554503DCA8
:1083600003FB0050012601E04FF0FF3614F8015BDB
:10837000D7E7731C0CD1002F4FF022030CBF6FF016
:1083800000404FF00040CCF800302AB9BDE8F08F33
:1083900007B1404242B106B1611E1160BDE8F08FE5
:1083A000002B08BF0823B0E7BDE8F08F7888FF1FD7
:1083B00030B51346044A05460C4610682946224645
:1083C000BDE83040FFF772BF7488FF1F2DE9F04110
:1083D000ADF5047D1D464FF400730F4690460393A0
:1083E000044618B183690BB900F094F804AE009507
:1083F0002046314603AA434600F05FF9054670B1B6
:10840000204639462A46039B00F01EF8B5420390E9
:1084100003D020462946FFF747FE039801E04FF0BE
:10842000FF300DF5047DBDE8F081FFFF30B5134648
:10843000044A05460C46106829462246BDE83040ED
:10844000FFF7C4BF7488FF1F38B5074C05460020EE
:108450002060084611461A46FFF730F9431C02D146
:10846000236803B12B6038BD1891FF1FF8B507468C
:1084700000F1480494B1A5686668013E0CD4AB894C
:10848000012B07D9B5F90E30013303D03846294600
:1084900000F0D6F96835F0E72468EBE7F8BDFFFF98
:1084A000002310B504460360436083608181436606
:1084B000C28103614361836119465C300822FFF782
:1084C000DDFD054B6362054BA362054BE362054B83
:1084D0002462236310BD00BF35860000578600006C
:1084E0008F860000B386000070B54B1E68255D4383
:1084F0000E4605F17401FFF71BFE044640B1002152
:1085000080E842000C30A06005F16802FFF7B6FD7C
:10851000204670BD836910B5044633BB8364C364D1
:108520000365124B124A1B688262984204BF012302
:10853000836100F01FF86060204600F01BF8A06027
:10854000204600F017F80421E06000226068FFF781
:10855000A7FFA06809210122FFF7A2FFE06812210E
:108560000222FFF79DFF0123A36110BD84B000002C
:108570006D840000F8B51B4B1E68B369074613B93C
:108580003046FFF7C7FF4836B4687368013B04D430
:10859000B4F90C5075B16834F8E733682BB9384634
:1085A0000421FFF7A1FF306008B13668ECE70C2327
:1085B0003B60F8BD4FF6FF73E3810123A38165663D
:1085C0002560A560656025616561A56104F15C00B9
:1085D00029460822FFF752FD6563A563A564E5649B
:1085E0002046F8BD84B00000F8B5064614460D4696
:1085F00021B91146BDE8F840FFF79ABD1AB9FFF757
:1086000053FD2046F8BD00F057F9A0420ED2304687
:108610002146FFF78DFD074650B129462246FCF75B
:10862000BBFA30462946FFF73FFD01E02846F8BD7A
:108630003846F8BD10B50C46B1F90E1000F046F9F9
:10864000002803DB636D0344636510BDA38923F435
:108650008053A38110BD2DE9F0411D468B89DB05B8
:1086600007460C46164605D5B1F90E100022022326
:1086700000F010F9A389B4F90E1023F48053A381FC
:10868000384632462B46BDE8F041FFF7DDBE10B557
:108690000C46B1F90E1000F0FDF8431CA38903D17C
:1086A00023F48053A38110BD43F48053A3816065FC
:1086B00010BDB1F90E1000F02FB830B515469BB0C3
:1086C000146829B124B14FF4C162ADF80C2005E063
:1086D0004FF422720024ADF80C202146002C0091AA
:1086E000049103DA8B230360002012E04FF6FF723F
:1086F000ADF80E2069461A461E9B0294059400F0C0
:1087000053F9031E4FF0000003DB2B60009B187031
:1087100004981BB030BDFFFF38B5064C002305465A
:1087200008462360FCF7FAFD431C02D1236803B11D
:108730002B6038BD1891FF1F8A892DE9F04105464D
:1087400010070C4657D44B68002B02DC0B6C002B37
:1087500018DDE66AB6B102F48052002392B22F68A7
:108760002B600AB1626D10E0216A28460123B047F0
:10877000411C024609D12B683BB11D2B01D0162BA1
:1087800046D12F600020BDE8F081A3895B0705D5A5
:108790006368D21A636B0BB1236CD21AE66A216A42
:1087A00028460023B047461CA28905D12B681BB17F
:1087B0001D2B01D0162B19D100236360D10423692E
:1087C000236004D5421C01D12B6803B96065616B3D
:1087D0002F600029D6D004F14403994202D02846E4
:1087E000FFF762FC00206063BDE8F08142F04002C8
:1087F000A281BDE8F0810E69002EC3D00B680E6027
:10880000C6EB030893070CBF4B6900238B6012E093
:10881000A38943F04003A3814FF0FF30BDE8F0810E
:10882000A76A216A284632464346B8470028EFDD4A
:108830000644C0EB0808B8F1000FF1DCA2E7FFFF27
:1088400038B50B6905460C46DBB118B183690BB925
:10885000FFF760FE0C4B9C4201D16C6808E00B4BAB
:108860009C4201D1AC6803E0094B9C4208BFEC6814
:10887000B4F90C302BB128462146BDE83840FFF74B
:108880005BBF002038BD00BF8CB10000ACB1000060
:10889000CCB1000038B5074C0546002020600846E2
:1088A00011461A46FCF73DFD431C02D1236803B173
:1088B0002B6038BD1891FF1F51F8040C002802DA14
:1088C00004390B58184404387047FFFF38B5074C7B
:1088D000054600202060084611461A46FCF71CFD9C
:1088E000431C02D1236803B12B6038BD1891FF1FD0
:1088F0002DE9F0478D68AB4281460C4692461F46F3
:1089000043D38B8913F4906F3DD026680969C1EB7E
:1089100006086669022206EB460696FBF2F608F1A7
:1089200001023A44964238BF16465B050FD53146E0
:10893000FFF7FEFB054698B121694246FCF72CF98A
:10894000A38923F4906343F08003A38113E03246AC
:10895000FFF74AFE054670B948462169FFF7A4FBB8
:108960000C23C9F80030A38943F04003A3814FF0E2
:10897000FF30BDE8F087256166614544C8EB060617
:108980002560A6603D46AF4200D23D462A4620689B
:108990005146FFF758FBA3685B1BA36023681D4487
:1089A00025600020BDE8F0872DE9F0439DB0074623
:1089B00003938B891C060D4616460CD50B6953B9DB
:1089C0004021FFF7B5FB2860286110B90C233B60FC
:1089D000C8E040236B610023099320238DF82930E0
:1089E00030238DF82A3033461C4613F8012B1AB970
:1089F000B4EB06090FD002E0252AF5D1F8E7384696
:108A0000294632464B46FFF773FF013000F0A58040
:108A1000099B4B4409932378002B00F09E80002390
:108A20004FF0FF3204930793059206938DF853306D
:108A30001A9304F101094C464D4E21783046052227
:108A4000FFF7F2FA09F10109049B28B1861B012006
:108A5000B04003430493EEE7D90644BF20228DF8CB
:108A600053201A0744BF2B228DF8532022782A2A3C
:108A700002D0079B21460EE0039A111D1268039154
:108A8000002A01DB079204E0524243F002030792FE
:108A9000049301340AE00C4601312278303A092A65
:108AA00003D80A2000FB0323F5E7079323782E2B36
:108AB0001AD163782A2B0AD1039B1A1D1B680392D3
:108AC000002B04F10204B8BF4FF0FF330BE0611C30
:108AD00000230C4601312278303A092A03D80A20B3
:108AE00000FB0323F5E70593224E2178304603224D
:108AF000FFF79AFA30B1861B049B4020B040034335
:108B00000493013421781C488DF828100622661C35
:108B1000FFF78AFA88B1194B33B9039B073323F067
:108B200007030833039314E003AB0093384604A90A
:108B30002A46134BAFF3008007E003AB009338469F
:108B400004A92A460E4B00F08FF8B0F1FF3F804693
:108B500003D0099B4344099345E7AB895B0601D4E5
:108B6000099801E04FF0FF301DB0BDE8F08300BF71
:108B7000ECB10000F2B10000F6B10000000000000E
:108B8000F18800002DE9F84315461F468A680B69F5
:108B9000DDF820809A42A8BF13462B6091F843204D
:108BA00006460C460AB101332B602368990602D5AC
:108BB0002B6802332B60236813F006091DD094F84C
:108BC00043302268003318BF012392061FD5E118F5
:108BD0005A1C302081F84300224494F8451082F852
:108BE0004310023313E03046394604F119020123E1
:108BF000C047013007D009F10109E2682B68D31A98
:108C00009945F0DBDBE74FF0FF30BDE8F8833046F5
:108C1000394604F14302C0470130F4D023682A6882
:108C2000E16803F00603042B08BFC2EB01052369CA
:108C3000A2680CBF25EAE57500259A42C4BFC3EBC4
:108C40000203ED184FF00009A9450ADA304639460B
:108C500004F11A020123C0470130D4D009F10109FF
:108C6000F2E70020BDE8F8832DE9FF470E7E0C9D5A
:108C70006E2E80460C4691469A4601F1430000F064
:108C8000A58011D8632E22D009D8002E00F0AF8025
:108C9000582E40F0BF8081F845607B4A4FE0642E3B
:108CA0001ED0692E1CD0B5E0732E00F0A48009D828
:108CB0006F2E2BD0702E40F0AD800B6843F0200358
:108CC0000B6038E0752E21D0782E34D0A2E02B68CE
:108CD0001A1D1B682A6001F1420781F842309DE0AD
:108CE00022682B6812F0800F03D01A1D2A601D68BD
:108CF00005E05106F9D51A1D2A60B3F90050002D80
:108D000039DA2D236D4284F8433034E022682B6831
:108D100012F0800F03D01A1D2A601D6804E052066D
:108D2000F9D51A1D2A601D88237E574A6F2B14BF60
:108D30000A2308231BE07823544A84F8453023682B
:108D4000296813F0800F01F104062E6001D00D6830
:108D500002E05F06FBD50D88DE0744BF43F0200329
:108D600023601DB9236823F0200323601023002112
:108D700084F8431001E0444A0A236668A660002E86
:108D800003DB216821F00401216005B96EB104F113
:108D90004201B5FBF3F603FB16550F46555D01F88E
:108DA00001593546002EF4D100E00746082B0AD1C0
:108DB0002368DD0707D5626823699A4203DC302304
:108DC00007F8013C013FC01B20612CE009682B68BB
:108DD000626911F0800F04D0191D29601B681A60A8
:108DE00005E04906F8D5191D29601B681A80002383
:108DF0002361074617E02B681A1D2A601F68384652
:108E0000FFF723FA63682061984288BF23612369D2
:108E1000636005E004F1420784F8426001232361A6
:108E2000002384F84330CDF800A04046214603AA31
:108E30004B46FFF7A7FE013002D14FF0FF301FE095
:108E4000404649463A462369D0470130F5D0236869
:108E50009B0705D4E068039B9842B8BF18460FE013
:108E60000025E268039BD31A9D42F3DA4046494647
:108E700004F119020123D0470130DED00135F0E7BB
:108E800004B0BDE8F08700BFFDB100000EB20000E5
:108E90005B4254204E4F542050524553454E545D32
:108EA0000041542B554152543D25642C302C300048
:108EB0000D0A004F4B0041540041542B4E414D458B
:108EC0003F0041542B505357443F005B4D41494EA6
:108ED0004252445F554E535550525445445D0041F3
:108EE000542B4E414D453D25730041542B50535753
:108EF000443D2530346900636C735F43697263429B
:108F000075666665725F3100636C734369726342B4
:108F100075666665725F320044756D70696E6720B4
:108F200043697263756C6172206275666665725F13
:108F3000006275666665725F2073697A6520697381
:108F40003A2025640A00252E32782000FFFFFFFF1B
:108F5000000000000000000029530000D5130000AD
:108F6000ED130000000000001801FFFFFFFFFFFFEE
:108F7000000000000000000015140000E1130000D4
:108F800001140000000000005B74696D656F75746A
:108F90005D0A005B25645D205B25645D0A005B70F3
:108FA0006172616D735F636F756E742025645D20FF
:108FB0005B25645D0A00556E6B6E6F776E2073746F
:108FC00061746520696E2063616C6C6261636B2003
:108FD000696E20636C73436F6E736F6C6521212122
:108FE0000A00496E69742064796E207061636B6554
:108FF000740050617274696C6C79206F70656E20BA
:1090000068616E642066756E6374696F6E616C6909
:109010007479206973206E6F742079657420696D8E
:10902000706C656D656E74656420696E2074686926
:1090300073206669726D77617265207665727369F7
:109040006F6E2E20504C65617365207573652074BA
:10905000686520636F6D6D616E6420746F20736549
:109060007420736572766F20706F736974696F6EA8
:109070007320696E646976696475616C6C792E0A17
:1090800000436C6F73652068616E642066756E6363
:1090900074696F6E616C697479206973206E6F7486
:1090A0002079657420696D706C656D656E7465649A
:1090B00020696E20746869732076657273696F6EBB
:1090C0002E205573652074686520636F6D6D616E29
:1090D0006420746F2073657420736572766F2070DE
:1090E0006F736974696F6E7320696E646976696401
:1090F00075616C6C792E0A005363616E6E696E67E0
:1091000020696E2070726F677265732E20557365CB
:1091100020636F6D6D616E64202773746174757365
:109120002720746F206C6973742049447320666F24
:10913000756E642E00596573004E6F00536565644B
:1091400020526F626F746963732045524F532046FB
:1091500069726D776172650A00426F617264206D99
:109160006F64656C2025640A00426F617264204858
:109170005720436F6E66696775726174696F6E2000
:1091800025640A004669726D7761726520766572A2
:1091900073696F6E2025640A0053657269616C20E3
:1091A0004E756D62657220252E3278252E32782517
:1091B0002E32780A0043757272656E742073656E84
:1091C000736F72207265736973746F722076616C4D
:1091D00075653A2025640A00426F617264206973E4
:1091E00020636F6E6669677572656420746F206FA7
:1091F00070657261746520776974682031326269C4
:1092000074207265736F6C7574696F6E2E0A0042FC
:109210006F61726420697320636F6E66696775722F
:10922000656420746F206F70657261746520776962
:109230007468203130626974207265736F6C757464
:10924000696F6E2E0A000A45787465726E616C2033
:1092500062757320636F6D6D756E69636174696F9C
:109260006E2073657474696E67733A200A00426FEA
:109270006172642062757320646576696365204954
:10928000443A2025640A0052657475726E20646544
:109290006C61792074696D653A202564205B2564D2
:1092A000206D6963726F736563735D0A0053746147
:1092B0007475732072657475726E206C6576656C5A
:1092C0003A2025640A005573696E6720545820457A
:1092D0006E61626C652070696E3A2025730A000A1F
:1092E000496E7465726E616C2062757320636F6D78
:1092F0006D756E69636174696F6E207365747469EE
:109300006E67733A20000A496E7465726E616C2054
:1093100062757320426175642072617465207365A3
:109320007474696E673A202564203D2025642042CC
:1093300050530A000A4120426C7565746F6F74685F
:1093400020636F6D6D756E69636174696F6E206DFA
:109350006F64756C652069732070726573656E74D7
:109360003A0A00426C7565746F6F746820434F4D04
:109370004D20426175642073657474696E672025A1
:1093800064203D202564204250530A00426C7565DC
:10939000746F6F746820646576696365206E616DB3
:1093A000653A202573200A00426C7565746F6F74EE
:1093B000682064657669636520636F64653A20257B
:1093C000303464200A000A4E6F20426C7565746F59
:1093D0006F746820636F6D6D756E69636174696F1A
:1093E0006E206D6F64756C6520646574656374656B
:1093F000642E0A004F6E004F666600426F61726411
:10940000205374617475733A0A00496E7465726E04
:10941000616C2054656D70657261747572653A098E
:10942000256420646567430A0045787465726E613F
:109430006C20537570706C7920566F6C7461676521
:109440003A0925642E2564560A00436F6E666967E3
:109450007572656420566F6C7461676520696E2053
:10946000496E7465726E616C204275733A092564A9
:10947000560A0A00506F736974696F6E2053656EE7
:10948000736F722057416464756374696F6E3A0933
:1094900025640A00506F736974696F6E2053656E9E
:1094A000736F722057466C6578696F6E3A09256450
:1094B0000A0050616C6D204F70746963616C2053B9
:1094C000656E736F7220696E7374616C6C65643A5B
:1094D0000925730A0050616C6D204F7074696361D7
:1094E0006C2053656E736F7220416D6269656E7496
:1094F000204C696768743A0925640A0050616C6DF4
:10950000204F70746963616C2053656E736F7220B5
:10951000436F6D70757465642052656164696E6730
:109520003A0925640A00436170616369746976656C
:109530002053656E736F727320696E7374616C6C07
:1095400065643A0925730A0043617061636974694F
:1095500076652053656E736F722031207265616489
:10956000696E673A0925640A004361706163697432
:109570006976652053656E736F7220322072656163
:1095800064696E673A0925640A000A436F6D6D7558
:109590006E69636174696F6E20537461746973746A
:1095A0006963733A0A005541525431202845787452
:1095B0002E436F6D6D2920427566666572204F7669
:1095C000657272756E733A2025640A0055415254D3
:1095D000322028496E742E436F6D6D2920427566C6
:1095E000666572204F76657272756E733A202564D7
:1095F0000A005541525433205B42542E436F6D6D27
:109600005D20427566666572204F76657272756E72
:10961000733A2025640A000A536572766F20494424
:109620007320696E2074686520496E7465726E617E
:109630006C204275733A0A000A506F72742073747A
:10964000617475733A0A00506F7274202564204368
:10965000757272656E742052656164696E673A2036
:109660004F5645524C4F4144204552524F522028AC
:1096700025646D41290A00506F72742025642043CF
:10968000757272656E742052656164696E673A2006
:1096900025646D410A000A4120426C7565746F6F44
:1096A000746820636F6D6D756E69636174696F6E48
:1096B000206D6F64756C65206973207072657365C9
:1096C0006E742E0A00426C7565746F6F746820703A
:1096D0006F776572207374617475733A2025730A0D
:1096E000005365656420526F626F7469637320452F
:1096F000524F53204669726D776172652C207665F2
:109700007273696F6E2025640A0A004C69737420B5
:109710006F6620616476616E63656420636F6D6D52
:10972000616E64732E0A5741524E494E473A205497
:109730006865736520636F6D6D616E64732061721F
:109740006520726573657276656420666F72207439
:10975000686520757365206F6620536565642052C7
:109760006F626F7469637320746563686E696361A7
:109770006C206167656E74732E0A496E636F727236
:10978000656374207573616765206D61792063611D
:1097900075736520696E6F7065726174696F6E2C88
:1097A0002064616D61676520616E64206D61792060
:1097B000766F696420796F75722077617272616E5D
:1097C00074792E0A55736520617420796F75722043
:1097D0006F776E207269736B2E0A0A0061687009D8
:1097E00054686973206D6573736167652E0A00693B
:1097F0006E697420656570726F6D0A00696E6974B8
:1098000020626F6172646D6F64656C205B6D6F6464
:10981000656C5D0A00696E697420626F61726468CC
:1098200077636F6E666967205B636F6E666967203A
:109830006D61736B5D0A00696E6974206375727285
:10984000656E747265736973746F72205B72657391
:109850006973746F722076616C7565204F686D73E3
:109860005D0A00696E697420736E205B59595D2032
:109870005B4D4D5D205B434845434B53554D5D0A61
:1098800000696E69742073657269616C636F6D6DD8
:10989000205B6C6566747C72696768745D0A0A0097
:1098A0005573652027636F6E6669672720666F7240
:1098B000207468652072656D61696E696E672063EA
:1098C0006F6E66696775726174696F6E732E20546E
:1098D000797065202768656C702720666F72206933
:1098E0006E666F726D6174696F6E2E0A0A004C6944
:1098F0007374206F6620617661696C61626C6520AB
:10990000636F6D6D616E64732E20416C6C20636FAC
:109910006D6D616E64732061726520636173652093
:1099200073656E7369746976652E0A0A0068656CE2
:10993000700954686973206D6573736167652E0AD9
:109940000073746174757309446973706C61792074
:1099500063757272656E742073797374656D2073AC
:1099600074617475732E0A0061626F7574094469BD
:1099700073706C617920696E7465726E616C2069B8
:109980006E666F726D6174696F6E2E0A007363612B
:109990006E6275730952657363616E7320746865D6
:1099A00020696E7465726E616C2062757320666FDB
:1099B000722044796E616D6978656C2064657669A2
:1099C0006365732E0A006F70656E094F70656E20B7
:1099D00068616E642E0A00636C6F736509436C6F77
:1099E00073652068616E642E0A00706172746F7016
:1099F000656E205B76616C75653A20302D25645D5F
:109A0000095061727469616C6C79206F70656E20A9
:109A100068616E642E0A00736574706F73205B64F6
:109A200065766963652069645D205B706F73697436
:109A3000696F6E3A20302D25645D0953657420707E
:109A40006F736974696F6E20666F722073706563DF
:109A50006966696564206465766963652E0A0072CB
:109A6000657374617274205B7073757C616C6C5D7E
:109A7000095265737461727473206F6E6C7920740F
:109A8000686520736572766F20505355206F722081
:109A90007468652066756C6C2073797374656D2EBF
:109AA0000A00636F6E666967205B65787462617532
:109AB000647C65787469647C6578747478656E61BB
:109AC000626C657C31326269746164636578706F61
:109AD0007365647C696E74626175647C62746261D2
:109AE00075647C62746E616D657C6274636F6465BD
:109AF0007C6274636F6D6D616E645D205B76616C1A
:109B000075655D0A0953797374656D2077696465BD
:109B100020636F6E66696775726174696F6E206F1E
:109B20007074696F6E732E0A00777262205B6465D1
:109B3000766963652069645D205B61646472657346
:109B4000735D205B627974652076616C75655D0973
:109B50005772697465206279746520746F2064653A
:109B6000766963652E0A00777277205B6465766993
:109B700063652069645D205B616464726573735D15
:109B8000205B696E742076616C75655D095772693A
:109B9000746520776F726420746F206465766963E2
:109BA000652E0A00726562205B64657669636520D4
:109BB00069645D205B616464726573735D095265FD
:109BC000616420627974652066726F6D20646576C9
:109BD0006963652E0A00726577205B646576696348
:109BE000652069645D205B616464726573735D09FF
:109BF0005265616420776F72642066726F6D2064B5
:109C000065766963652E0A0A00496E76616C69643F
:109C100020636F6D6D616E642E20436F6D6D616E9C
:109C200064732061726520636173652073656E7370
:109C300069746976652E0A54797065202768656CA9
:109C4000702720666F72206D6F726520696E666F77
:109C5000726D6174696F6E2E0A004944206E6F74D4
:109C60002070726573656E7420696E20746865205B
:109C7000696E7465726E616C206275732E20547902
:109C8000706520277374617475732720666F722066
:109C900061206C697374206F662076616C69642042
:109CA0004944732E0A00496E76616C696420706FB6
:109CB000736974696F6E2E204D6178696D756D20C2
:109CC000616363657074656420706F736974696F34
:109CD0006E20697320343039352E0A416374756102
:109CE0006C206D6178696D756D20646570656E645A
:109CF00073206F6E206163747561746F7220636F7F
:109D00006E66696775726174696F6E2E0A00707392
:109D10007500446F6E6500616C6C006578747478D2
:109D2000656E61626C6500796573006E6F0031323B
:109D30006269746164636578706F73656400696EED
:109D400074626175640062746261756400496E7664
:109D5000616C69642073657474696E672E20536545
:109D60007474696E672073686F756C642062652017
:109D700061204261756420706172616D6574657205
:109D800020286578616D706C653A2031363D31313F
:109D900035323030627073290053756365737320F8
:109DA000636F6E6669677572696E67204254206DD5
:109DB0006F64756C652E0A004661696C656420638A
:109DC0006F6E6669677572696E67204254206D6FA9
:109DD00064756C652E0A0053617665642073657442
:109DE00074696E6720696E204D61696E20626F61D3
:109DF000726420656570726F6D2E0062746E616DA5
:109E000065005375636573730A004661696C0A00E7
:109E10006274636F646500496E76616C6964206387
:109E20006F64652E20436F6465206D7573742062C6
:109E30006520612034206469676974206E756D65E2
:109E400072696320636F64652072616E67696E6713
:109E50002066726F6D203030303020746F203939B9
:109E600039392E0A00537563636573732E2042548B
:109E700020636F64652073657420746F20272573D9
:109E8000272028616C776179732061203420646910
:109E900067697420636F6465292E0A006274636FBA
:109EA0006D6D616E64005265706C793A0A25730AB3
:109EB00000656570726F6D00626F6172646D6F64D2
:109EC000656C00626F6172646877636F6E66696764
:109ED0000063757272656E747265736973746F7204
:109EE0000073657269616C636F6D6D006C6566749B
:109EF00000726967687400736E0068656C70006159
:109F00006870007374617475730061626F757400BA
:109F10007363616E62757300636C6F73650070616B
:109F200072746F70656E00736574706F7300726524
:109F30007374617274007772620077727700726571
:109F4000620072657700466978656453697A654492
:109F5000786C436F6D6D616E645175657565004613
:109F60006978656453697A6544786C436F6D6D6197
:109F70006E6451756575655F62797465736172723F
:109F8000617900466978656453697A6544786C4301
:109F90006F6D6D616E6451756575655F6269646949
:109FA000726C697374000A44554D50204C495354E7
:109FB0000A004865616420616464722025702C2069
:109FC0005461696C20616464722025702C2049748E
:109FD000656D20636F756E742025642C207074721B
:109FE000206469666572656E63652025640A0041B8
:109FF0006464722025702C20536572766F2049446A
:10A000002025640A00636C735F4D61696E426F6165
:10A0100072645F696E697400000000000000000057
:10A02000153E00001D3700004D3700000000000005
:10A030000000000000000000094000009D3E0000FC
:10A04000C53E0000D73E0000253F0000713F0000E4
:10A05000B93F00001B420000A143000000000000C7
:10A0600000000000000000002953000081440000AF
:10A07000A94400002953000029530000295300007F
:10A08000295300002953000029530000000000005C
:10A0900000000000010000000200000003000000BA
:10A0A0000400000006000000070000000800000097
:10A0B000090000000A0000000B0000000C00000076
:10A0C0000D0000000E0000000F0000001000000056
:10A0D0001100000012000000130000001400000036
:10A0E0001500000016000000180000001900000014
:10A0F0001A0000001B0000001C0000001D000000F2
:10A100001E0000001F0000002000000021000000D1
:10A1100022000000230000002400000025000000B1
:10A120002600000027000000280000002900000091
:10A130002A0000002B0000002C0000002D00000071
:10A140002E0000002F000000300000003100000051
:10A150003200000033000000340000003500000031
:10A160003600000037000000380000003900000011
:10A170003A0000003B0000003C0000003D000000F1
:10A180003E0000003F0000004000000041000000D1
:10A1900042000000430000004400000044000000B2
:10A1A0004500000046000000470000004800000095
:10A1B000490000004A0000004B0000004C00000075
:10A1C0004D0000004E0000004F0000005000000055
:10A1D0005100000052000000530000005400000035
:10A1E0005500000056000000570000005800000015
:10A1F00058000000590000005A0000005B000000F9
:10A200005C0000005D0000005E0000005F000000D8
:10A2100060000000610000006200000063000000B8
:10A220006400000065000000660000006600000099
:10A230006700000068000000690000006A0000007C
:10A240006B0000006C0000006D0000006E0000005C
:10A250006F0000007000000071000000720000003C
:10A260007200000073000000740000007500000020
:10A270007600000077000000780000007900000000
:10A280007A0000007B0000007C0000007C000000E1
:10A290007D0000007E0000007F00000080000000C4
:10A2A00081000000820000008300000084000000A4
:10A2B0008500000086000000860000008700000086
:10A2C00088000000890000008A0000008B00000068
:10A2D0008C0000008D0000008E0000008F00000048
:10A2E0008F0000009000000091000000920000002C
:10A2F000930000009400000095000000960000000C
:10A3000097000000970000009800000099000000EE
:10A310009A0000009B0000009C0000009D000000CF
:10A320009E0000009F0000009F000000A0000000B1
:10A33000A1000000A2000000A3000000A400000093
:10A34000A5000000A6000000A7000000A700000074
:10A35000A8000000A9000000AA000000AB00000057
:10A36000AC000000AD000000AE000000AF00000037
:10A37000AF000000B0000000B1000000B20000001B
:10A38000B3000000B4000000B5000000B6000000FB
:10A39000B6000000B7000000B8000000B9000000DF
:10A3A000BA000000BB000000BC000000BD000000BF
:10A3B000BE000000BE000000BF000000C0000000A2
:10A3C000C1000000C2000000C3000000C400000083
:10A3D000C5000000C5000000C6000000C700000066
:10A3E000C8000000C9000000CA000000CB00000047
:10A3F000CC000000CD000000CD000000CE00000029
:10A40000CF000000D0000000D1000000D20000000A
:10A41000D3000000D4000000D4000000D5000000EC
:10A42000D6000000D7000000D8000000D9000000CE
:10A43000DA000000DB000000DC000000DC000000AF
:10A44000DD000000DE000000DF000000E000000092
:10A45000E1000000E2000000E3000000E400000072
:10A46000E4000000E5000000E6000000E700000056
:10A47000E8000000E9000000EA000000EB00000036
:10A48000EB000000EC000000ED000000EE0000001A
:10A49000EF000000F0000000F1000000F2000000FA
:10A4A000F3000000F3000000F4000000F5000000DD
:10A4B000F6000000F7000000F8000000F9000000BE
:10A4C000FA000000FB000000FC000000FC0000009F
:10A4D000FD000000FE000000FF0000000001000081
:10A4E000010100000201000003010000040100005E
:10A4F0000401000005010000060100000701000042
:10A5000008010000090100000A0100000B01000021
:10A510000C0100000D0100000D0100000E01000003
:10A520000F010000100100001101000012010000E5
:10A5300013010000140100001501000016010000C5
:10A5400017010000170100001801000019010000A8
:10A550001A0100001B0100001C0100001D01000089
:10A560001E0100001F010000200100002101000069
:10A57000210100002201000023010000240100004D
:10A58000250100002601000027010000280100002D
:10A59000290100002A0100002B0100002C0100000D
:10A5A0002D0100002D0100002E0100002F010000F0
:10A5B00030010000310100003201000033010000D1
:10A5C00034010000350100003601000037010000B1
:10A5D00038010000390100003A0100003B01000091
:10A5E0003B0100003C0100003D0100003E01000075
:10A5F0003F01000040010000410100004201000055
:10A600004301000044010000450100004601000034
:10A610004701000048010000490100004A01000014
:10A620004B0100004C0100004D0100004E010000F4
:10A630004F0100004F0100005001000051010000D7
:10A6400052010000530100005401000055010000B8
:10A650005601000057010000580100005901000098
:10A660005A0100005B0100005C0100005D01000078
:10A670005E0100005F010000600100006101000058
:10A680006201000063010000640100006501000038
:10A690006601000067010000680100006901000018
:10A6A0006A0100006B0100006C0100006D010000F8
:10A6B0006E0100006F0100007001000071010000D8
:10A6C00072010000730100007401000075010000B8
:10A6D0007601000077010000780100007901000098
:10A6E0007A0100007B0100007C0100007D01000078
:10A6F0007E0100007F010000800100008101000058
:10A700008201000083010000840100008501000037
:10A710008601000088010000890100008A01000014
:10A720008B0100008C0100008D0100008E010000F3
:10A730008F010000900100009101000092010000D3
:10A7400093010000940100009501000096010000B3
:10A7500097010000980100009A0100009B01000091
:10A760009C0100009D0100009E0100009F0100006F
:10A77000A0010000A1010000A2010000A30100004F
:10A78000A4010000A6010000A7010000A80100002C
:10A79000A9010000AA010000AB010000AC0100000B
:10A7A000AD010000AE010000B0010000B1010000E9
:10A7B000B2010000B3010000B4010000B5010000C7
:10A7C000B6010000B7010000B9010000BA010000A5
:10A7D000BB010000BC010000BD010000BE01000083
:10A7E000C0010000C1010000C2010000C30100005F
:10A7F000C4010000C5010000C7010000C80100003D
:10A80000C9010000CA010000CB010000CC0100001A
:10A81000CE010000CF010000D0010000D1010000F6
:10A82000D2010000D4010000D5010000D6010000D3
:10A83000D7010000D8010000DA010000DB010000B0
:10A84000DC010000DD010000DF010000E00100008C
:10A85000E1010000E2010000E4010000E501000068
:10A86000E6010000E7010000E9010000EA01000044
:10A87000EB010000EC010000EE010000EF01000020
:10A88000F0010000F2010000F3010000F4010000FB
:10A89000F5010000F7010000F8010000F9010000D7
:10A8A000FB010000FC010000FD010000FF010000B1
:10A8B0000002000001020000030200000402000088
:10A8C0000502000007020000080200000902000063
:10A8D0000B0200000C0200000D0200000F0200003D
:10A8E0001002000012020000130200001402000017
:10A8F0001602000017020000190200001A020000F0
:10A900001B0200001D0200001E02000020020000C9
:10A9100021020000230200002402000026020000A1
:10A9200027020000280200002A0200002B0200007B
:10A930002D0200002E020000300200003102000053
:10A94000330200003402000036020000370200002B
:10A95000390200003A0200003C0200003E02000002
:10A960003F020000410200004202000044020000D9
:10A970004502000047020000490200004A020000B0
:10A980004C0200004D0200004F0200005102000086
:10A99000520200005402000056020000570200005C
:10A9A000590200005B0200005C0200005E02000031
:10A9B0006002000061020000630200006502000006
:10A9C00066020000680200006A0200006C020000DB
:10A9D0006D0200006F0200007102000073020000AF
:10A9E0007402000076020000780200007A02000083
:10A9F0007C0200007E0200007F0200008102000055
:10AA00008302000085020000870200008902000026
:10AA10008B0200008D0200008E02000090020000F8
:10AA200092020000940200009602000098020000CA
:10AA30009A0200009C0200009E020000A00200009A
:10AA4000A2020000A4020000A6020000A80200006A
:10AA5000AB020000AD020000AF020000B102000036
:10AA6000B3020000B5020000B7020000B902000006
:10AA7000BC020000BE020000C0020000C2020000D2
:10AA8000C4020000C7020000C9020000CB0200009F
:10AA9000CE020000D0020000D2020000D502000069
:10AAA000D7020000D9020000DC020000DE02000034
:10AAB000E1020000E3020000E5020000E8020000FD
:10AAC000EA020000ED020000F0020000F2020000C5
:10AAD000F5020000F7020000FA020000FC0200008C
:10AAE000FF0200000203000005030000070300004E
:10AAF0000A0300000D030000100300001203000011
:10AB000015030000180300001B0300001E030000D3
:10AB10002103000024030000270300002A03000093
:10AB20002D03000030030000330300003603000053
:10AB3000390300003D030000400300004303000010
:10AB4000460300004A0300004D03000050030000CC
:10AB500054030000570300005B0300005E03000085
:10AB60006203000065030000690300006D0300003C
:10AB70007103000074030000780300007C030000F0
:10AB80008003000084030000880300008C030000A1
:10AB90009003000094030000980300009D03000050
:10ABA000A1030000A5030000AA030000AE030000FB
:10ABB000B3030000B8030000BC030000C1030000A1
:10ABC000C6030000CB030000D0030000D503000043
:10ABD000DA030000DF030000E5030000EA030000E1
:10ABE000EF030000F5030000FB0300000004000079
:10ABF000060400000C040000120400001904000008
:10AC00001F040000250400002C0400003304000091
:10AC10003A04000040040000480400004F04000013
:10AC2000560400005E040000660400006E0400008C
:10AC3000760400007E0400008704000090040000F9
:10AC400099040000A2040000AC040000B604000057
:10AC5000C0040000CA040000D5040000E0040000A5
:10AC6000EC040000F80400000405000011050000D9
:10AC70001E0500002C0500003A05000049050000F3
:10AC800059050000690500007A0500008C050000E8
:10AC90009F050000B3050000C8050000DE050000A8
:10ACA0004D616C6C6F63206661696C656420666FD2
:10ACB000722025730A005061636B65743A2000307E
:10ACC0007846462030784646203078004545505238
:10ACD0004F4D2077726974652064656E69656420E4
:10ACE000627920696E7465726E616C2070726F7427
:10ACF000656374696F6E2E204E72206F66207772C6
:10AD00006974657320617474656D7074656420691D
:10AD10006E20746869732073657373696F6E3A206F
:10AD200000417474656D7074696E6720746F20776C
:10AD300072697465206120424954206F6E20612041
:10AD40006269746D61702062757420697427732064
:10AD50006F7574206F662072616E67653B20746842
:10AD60006520616C6C6F7765642072616E67652029
:10AD7000697320307E372E00090AFFFFFFFFFFFFB7
:10AD8000FFFFFFFFFFFFFF0D00060807FFFF0E0F8D
:10AD9000FF0CFFFFFFFFFFFF0B05050E08090D0C61
:10ADA00006070F04001303931A9217C5858486873C
:10ADB000C4FF6FF07F030370037813F0800FFBD0A4
:10ADC0007047FFFF4008FE4340A004404408FE4394
:10ADD00044A004400018FE4300C004403000FE437D
:10ADE000309004403400FE43349004401C18FE436D
:10ADF0001CC004401018FE4310C004400818FE4355
:10AE000008C004400C18FE430CC004400C10FE4364
:10AE10000CB004401010FE4310B004401810FE4364
:10AE200018B004401C10FE431CB004401410FE4334
:10AE300014B004400418FE4304C004400010FE4354
:10AE400000B004400008FE4300A004400408FE4394
:10AE500004A004400C08FE430CA004400808FE4374
:10AE600008A004401418FE4314C004401818FE4300
:10AE700018C004400410FE4304B004400810FE4310
:10AE800008B004401400FE43149004404C08FE43F4
:10AE90004CA004400420FE4304D004402410FE4390
:10AEA00024B004402010FE4320B004402810FE438C
:10AEB00028B004402C10FE432CB004400020FE4378
:10AEC00000D004404808FE4348A004401000FE4360
:10AED00010900440090AFFFFFFFFFFFFFFFFFFFF85
:10AEE000FFFFFF0D00060807FFFF0E0FFF0CFFFF1F
:10AEF000FFFFFFFF0B05FFFF000000000000000048
:10AF0000DD730000F5730000C5730000CD73000011
:10AF1000C9730000D1730000697300007B730000E7
:10AF20009B7300009F730000A5730000B5730000C1
:10AF3000D5730000D9730000397300004573000019
:10AF4000517300005D73000005740000E973000098
:10AF50000000000000000000E1740000F97400002F
:10AF6000C9740000D1740000CD740000D5740000D5
:10AF70006D7400007F7400009F740000A3740000D3
:10AF8000A9740000B9740000D9740000DD740000D9
:10AF90003D740000497400005574000061740000A5
:10AFA00009750000ED7400000000000000000000C2
:10AFB000E5750000FD750000CD750000D575000039
:10AFC000D1750000D975000071750000837500000F
:10AFD000A3750000A7750000AD750000BD750000E9
:10AFE000DD750000E1750000417500004D75000041
:10AFF00059750000657500000D760000F1750000C0
:10B000000D0AFFFFFFFFFFFF00000000000000002F
:10B01000737700007977000063770000677700009E
:10B020006B7700006F770000001519150001000014
:10B030007487FF1F12000000000200009E87FF1FA0
:10B040004300000000030000F887FF1F000000001D
:10B05000010309048687FF1F0000000002030904A2
:10B06000E287FF1F0000000003030904FC87FF1FA5
:10B0700000000000000000000000000000000000D0
:10B080004300FFFF1488FF1F0020202020202020E5
:10B090002020282828282820202020202020202088
:10B0A0002020202020202020208810101010101098
:10B0B00010101010101010101004040404040404E4
:10B0C000040404101010101010104141414141417E
:10B0D0000101010101010101010101010101010160
:10B0E0000101010110101010101042424242424270
:10B0F0000202020202020202020202020202020230
:10B1000002020202101010102000000000000000D7
:10B11000000000000000000000000000000000002F
:10B12000000000000000000000000000000000001F
:10B13000000000000000000000000000000000000F
:10B1400000000000000000000000000000000000FF
:10B1500000000000000000000000000000000000EF
:10B1600000000000000000000000000000000000DF
:10B1700000000000000000000000000000000000CF
:10B18000000000000000000000FFFFFF00000000C2
:10B1900000000000000000000000000000000000AF
:10B1A000000000000000000000000000000000009F
:10B1B000000000000000000000000000000000008F
:10B1C000000000000000000000000000000000007F
:10B1D000000000000000000000000000000000006F
:10B1E000000000000000000000000000232D302BB4
:10B1F0002000686C4C006566674546470030313278
:10B2000033343536373839414243444546003031CE
:10B21000323334353637383961626364656600FF2E
:10B22000F8B500BFF8BC08BC9E4670473504000066
:10B230002174000025750000297600008577000044
:10B24000010000000A0400001C91FF1F080000001C
:10B25000FFFFFFFF1201000202000040C01683043E
:10B2600000010102030118035400650065006E002F
:10B27000730079006400750069006E006F000902B8
:10B280004300020100C03209040000010202010073
:10B2900005240010010524010101042402060524EF
:10B2A0000600010705820310004009040100020A9C
:10B2B000000000070503024000000705840240006B
:10B2C00000001603550053004200200053006500A3
:10B2D0007200690061006C00040309040C030000A3
:10B2E000000000000000000000000000000000005E
:10B2F00000000000000000008CB10000ACB10000B4
:10B30000CCB10000000000000000000000000000C0
:10B310000000000080B000000000000000000000FD
:10B32000000000000000000000000000000000001D
:10B33000000000000000000000000000000000000D
:10B3400000000000000000000000000000000000FD
:0CB35000000000001488FF1F88B00000FF
:00000001FF
